:0A00000075817F7401F58F02002E58
:03000B000202905E
:03002300026C82EA
:10002B0002022E7400900080F0900081F0743E90DC
:10003B000082F07400900083F0900084F0900085B3
:10004B00F0900086F0900087F07406900091F0A37A
:10005B00F07402900093F07402900094F07474901A
:10006B000095F07402900096F07407900097F0746E
:10007B003F900098F0A3F0A3F090009BF0A3F0A3A7
:10008B00F090009EF0A3F0A3F074079000A1F07421
:10009B00009000A2F09000A3F09000A4F0740190E7
:1000AB0000A5F09000A6F074009000A7F09000A8B7
:1000BB00F09000A9F09000AEF0A3F0A3F0A3F090A5
:1000CB0000AAF0A3F0A3F0A3F0120CCB853D3E12D7
:1000DB000CDC753F82753B00753C00C208D2107575
:1000EB005100D20DC21D757105757201757301C278
:1000FB0059C260C261C262C263C264D2167554191E
:10010B00755800755900C211C212C213C265C2667E
:10011B00C267C268C26912708C854F4A85504B7595
:10012B005B00755C00755D00755E00755F0075604A
:10013B00007561007562007563007564007565007C
:10014B007566007567007568001213D612145F127E
:10015B0014287A01121428120D91126C29120D32E7
:10016B00120EB8120ED21203D31202AC1202AC1240
:10017B0002AC1202AC1202ACC20BC208D20AC20C05
:10018B00C209755200755300757E01C220C221C28F
:10019B0022C223C224C225C226C227C228C229C218
:1001AB002AC22BC22CC22DC22EC22FC230C231C2C8
:1001BB0032C233C234C235C236C237C238C239C278
:1001CB003AC23BC23CC23DC23EC23FC240C241C228
:1001DB0042C243C244C245C246C247C248C249C2D8
:1001EB004AC24BC24CC24DC24EC24FD21AC21BD2D4
:1001FB001CD250D251D252D253D254D255D256D203
:10020B0057757600757700754E001202C0120458B0
:10021B009000F1E0B401061214AB020222125BBC97
:10022B00020228C0E0C0D0E582C0E0E583C0E0E96F
:10023B00C0E0EAC0E0EBC0E0120D681212B0D54787
:10024B002E754704120CCB120CDCD54822754805D1
:10025B00120F86D54919754932D204D54C11754CFC
:03026B0002C204C8
:10026E00054ED54D07754D03D215B26AD0E0FBD0C1
:10027E00E0FAD0E0F9D0E0F583D0E0F582D0D0D02E
:10028E00E032C0E0C0D0C2CFD54A0E754AFFD54B82
:10029E0008854F4A85504BD206D0D0D0E03278FF39
:1002AE0079FF0000D9FCD8F82278FF799BD9FED8C7
:1002BE00FA22756780120EECE569F4547F30E50D75
:1002CE0075670043628043638012033722E54EB4A4
:1002DE0003E0120F067567001202AC1202AC120296
:1002EE00AC1202AC1202AC1202AC125A389000F1EF
:1002FE00E0B40116120F131202AC1202AC1202ACD1
:10030E001202AC1202AC1202AC22120F20125C9E30
:10031E00E5740490007E12147D1202AC1202AC122F
:10032E0002AC1202AC1202AC22E569F4547F30E04A
:10033E003B74019000F1F0125A2453627F53637F95
:10034E00120EB890074005A29000667B04120EC4F0
:10035E001202AC1202AC120F131202AC1202AC1249
:10036E0002AC1202AC1202AC1202AC2230E14774A3
:10037E00029000F1F0125A2453627F53637F120EE3
:10038E00B890074005A29000667B04120EC41202BC
:10039E00AC1202AC120F20125C9EE5740490007E2B
:1003AE0012147D1202AC1202AC1202AC1202AC128A
:1003BE0002AC1202AC22206A06120EEC02033712B5
:1003CE000EDF020337755BFF7560FF756121120248
:1003DE00B7755CFF755FFF7561331202B7755DFF10
:1003EE00755EFF75613F1202B7755D00755E007533
:1003FE0061337564FF7565FF75680C1202B7755C25
:10040E0000755F007561217563FF7566FF75681E67
:10041E001202B7755B007560007561007562FF753D
:10042E0067FF75683F1202B77562007567007568E1
:10043E001E1202B775630075660075680C1202B75E
:10044E00756400756500756800229000F1E0B401D6
:10045E000712583F12047322B402FD754E00125C4F
:10046E00D41204AC22120EB8C21FC258756100120B
:10047E0038BA12316212325D1234E612347F7406CB
:10048E009000B5F01233867568205361FE4360808C
:10049E00227401900000F0757400125C8A22757F40
:1004AE0000C277C25F74789000F2F0C220C221C2FF
:1004BE0022C223C224C225C226C227C228C229C2F2
:1004CE002AC22BC22CC22DC22EC22FC230C231C2A2
:1004DE0032C233C234C235C236C237C238C239C252
:1004EE003AC23BC23CC23DC23EC23FC240C241C202
:1004FE0042C243C244C245C246C247C248C249C2B2
:10050E004AC24BC24CC24DC24EC24FC250C251C261
:07051E0052C253C254C25542
:10052500C256C257C214120EB8E57424B0126C7AC2
:10053500746D126C7A747F126C7A2203002C0C0194
:10054500057E2133E6FF0B4D68146405150D5A4BE6
:100555001B26351E1A96114042C8D520202046205C
:100565004C2041204D204520202020202053495853
:100575002D494E2D412D524F5720202020763120D8
:10058500323030382D323030392020313A20204D6C
:100595004944492D5048524153452D2020202020C3
:1005A50053455155454E4345522020323A20204D62
:1005B5004944492D52454D4F5445205048524153C9
:1005C500452D53455155454E43455220205665729C
:1005D50073696F6E20312E3030202020202863294A
:1005E500323030382D3230303920204D4944492DB4
:1005F50052454D4F54452D554E495420202020201D
:1006050056312E30322020202020204D4944492DBE
:100615004348414E4E454C3A2020205052455353B5
:10062500204B455920464F52204F4B464F522045AF
:10063500444954204348414E4E454C504C45415346
:1006450045205052455353204B4559494E49542056
:10065500414C4C2044415441203F20504C4541538E
:1006650045205052455353204B455920204F4B218F
:100675002020202043414E43454C21202020504C32
:1006850045415345205741495420205748494C4539
:1006950020494E495449414C495A45202020204182
:1006A5004C4C204441544120212020504C4541537D
:1006B50045205052455353204B4559202020544F37
:1006C5002053454C454354204120202020202050D4
:1006D500524F4752414D2021202020504C45415337
:1006E50045205052455353204B455920464F5220E3
:1006F50053454C454354494E4720205448452050C6
:10070500524F4752414D205041474520202020203F
:10071500204E4F5720202020202020544845204C93
:100725004153542050524F4752414D2020495320A8
:100735004C4F4144494E47202120204F4B20215208
:10074500616E646F6D205245414459202120504C03
:10075500454153452057414954202120202043231A
:100765004320442344204520462346204723472051
:1007750041234120422D322D31302031203220338A
:1007850020342035203620372038202020202020F6
:1007950020202020202020202020204D454C4F3A8D
:1007A50031202020202020202020204452554D207B
:1007B50020412020422020432020205345545550DD
:1007C500205041474520202020202054454D5030C1
:1007D5003A56454C4F434954593A5343414C453A8F
:1007E5004B45594E4F54453A43484F52443A504869
:1007F500524153453A415250454747494F3A424580
:1008050041543A4E4F54453A53494E474C45204E74
:100815004F5445202020202043484F52444E4F54EA
:1008250045534152502B4D494449434C4F434B3A54
:10083500696E7465726E4D494449204348414E4E78
:10084500454C3A3130204D656C6F64792D314D65DD
:100855006C6F64792D324472756D2D412020447280
:10086500756D2D4220204472756D2D4320206578CD
:100875007465726E53454E44434C4F434B3A6F6E0D
:10088500206F6666534156452055534552204441D5
:0E0895005441202050555420424C494E4B49AE
:1008A3004E47204B455953415645205041545445DA
:1008B300524E2F414C4C446F776E202020557020B0
:1008C300202020204F63746176652054726961642F
:1008D30020726F6F7454726961642031696E76544B
:1008E300726961642032696E764F637461766573F1
:1008F30020202052616E646F6D202020206E6F7265
:100903006D616C2020202F326E6F726D616C202020
:10091300202F346E6F726D616C2020202F386E6F24
:10092300726D616C20202F31366E6F726D616C2099
:10093300202F33326F66666265617420202F326F19
:1009430066666265617420202F346F666662656136
:100953007420202F386F666662656174202F3136EC
:1009630073687566666C6531202F387368756666C3
:100973006C6532202F3873687566666C6533202F7B
:100983003873687566666C65202F3136206C61722A
:10099300676F202061646167696F616E64616E7463
:1009A300656D6F6465726174616C6C6567726F20ED
:1009B3007669766163652070726573746F207072F7
:1009C30065737469747269706C6574080002030559
:1009D3000607080B000600010405070800000005D0
:1009E3000001030708000000000600030407090ACA
:1009F3000000000600030506070A000000070001C7
:100A0300040507080B0000050002040709000000A5
:100A130000070002030509060A0000070002040597
:100A230007080A0000070002040607090B00000775
:100A33000002040507090B00000400040709000075
:100A4300000000040004070B000000000004000481
:100A5300060A0000000000070002030507080A0059
:100A63000004000307090000000000040003070A54
:100A73000000000000070002030507080B00000741
:100A83000002040507090A0000090002030406071F
:100A930008090B08000103040607090A0005000200
:100AA30005070900000000070001030507080A0005
:100AB30000070001040507080A00000600020406F7
:100AC300080A0000000C00010203040506070809D8
:100AD3000A0B416C67657269616E20204172616225
:100AE30069616E20202042616C696E657365202008
:100AF300426C756573206D616A20426C7565732065
:100B03006D696E2042797A616E74696E65204469FD
:100B130061746F6E69632020446F7269616E202077
:100B2300202048696E647520202020204C79646958
:100B3300616E202020204D616A6F722020202020CA
:100B43004D616A6F7220362020204D616A6F7220DA
:100B5300372020204D616A6F7220372062354D693E
:100B63006E6F7220202020204D696E6F7220362018
:100B730020204D696E6F7220372020204D696E6FE3
:100B830072206861726D4D69786F6C796469616E0A
:100B93004E696E6520546F6E65204F637461746F88
:100BA3006E69632050656E7461746F6E696350681B
:100BB30072796769616E20205370616E6973682072
:100BC300202057686F6C65746F6E65204368726F81
:100BD3006D6174696320800080808888AAAAFFFF02
:100BE3000080080822225555848482828181999944
:100BF30088008200220008800220008820800820CC
:100C03000082000A000800028808882082208A00E7
:0E0C1300A080A00820882802220808A00882DD
:100C2100088888A882828A88A0A0AA0828280A0A97
:100C3100082AA2A222A2A280228082A2888A882ACD
:100C41008A0AA222A8A0A0A82A28222A282A0A8A37
:100C510008AAA2822282A08AA822A28AA8A2AA28DD
:100C61002ACA000C000F00F000F23234C8C8C8CA0A
:100C7100C88A8ECBAAD5A9A9CA98CE82CAE25959E7
:100C810033838F0A8DEAE2A2E82EF0F2BC3CF08CAD
:100C9100E4F2ABABBABAADADD6D6AFCAAAF8AACF19
:100CA100CF3FEEEEBB2CBBBBFF08FC8888FF0AFFE1
:100CB10000FF924882088200800802080248909052
:100CC100C30CDB08DB6FE38EE388209504753D00E0
:100CD10022209603D20322753D0122E53DB53E0453
:100CE100853D3E22B4001520030A053F853D3ED2D5
:100CF10005D20E22C203853D3ED2052220030A15EC
:100D01003F853D3ED205D20F22C203853D3ED2052D
:100D110022300503300406E53F1214922205A29009
:100D2100079005A27B03120EC422209703C205225D
:100D310022753A00C200C2B4C2B39000507439F0B7
:100D4100A3741DF0A37450F0A3746CF0A37479F034
:100D5100A3740FF0A37401F0A37406F0E53AB4088C
:100D6100FB753A00D20022E53AB4300DC2B375A04A
:100D710080D2B2C2B2753A0022A20092B390005062
:100D8100E582253AF582E0F5A0D2B2C2B2053A2257
:100D9100C2B4C2B375A040D2B2C2B21202B7D2B3CA
:100DA10075A000D2B2C2B21202B7D2B375A01ED2E0
:100DB100B2C2B21202B7D2B375A01ED2B2C2B2127F
:100DC10002B7D2B375A01ED2B2C2B21202B7D2B369
:100DD10075A01ED2B2C2B21202B7D2B375A01ED292
:100DE100B2C2B21202B7D2B375A01ED2B2C2B2124F
:100DF10002B7C2B4C2B375A048D2B2C2B21202B72E
:100E0100D2B375A000D2B2C2B21202B7D2B375A0EA
:100E110004D2B2C2B21202B7D2B375A00CD2B2C21E
:100E2100B21202B7D2B375A01CD2B2C2B21202B7CB
:100E3100D2B375A00CD2B2C2B21202B7D2B375A0AE
:100E410004D2B2C2B21202B7D2B375A000D2B2C2FA
:100E5100B21202B7C2B4C2B375A050D2B2C2B212BA
:100E610002B7D2B375A000D2B2C2B21202B7D2B3E6
:100E710075A010D2B2C2B21202B7D2B375A018D205
:100E8100B2C2B21202B7D2B375A01CD2B2C2B212B0
:100E910002B7D2B375A018D2B2C2B21202B7D2B39E
:100EA10075A010D2B2C2B21202B7D2B375A000D2ED
:100EB100B2C2B21202B72274209000507830F0A36F
:100EC100D8FC2205A2E493A305A2F0A3DBF505A2B9
:100ED1002290056005A29000507B30020EC490055F
:100EE1009005A29000507B30020EC49006B005A27E
:100EF1009000507B30020EC49006E005A290005095
:100F01007B30020EC490071005A29000507B300286
:100F11000EC49005C005A29000507B30020EC49013
:100F210005F005A29000507B30020EC4900610051A
:100F3100A29000607B20020EC490063005A29000B2
:100F4100607B20020EC4E53B053B900F4F73020FFF
:100F5100C6020FE5021004021023021042021061C2
:100F610002108002109F753B0022020FC6020FE59E
:100F71000210040210230210420210610210807557
:100F81003B0002109FE53BB40005053B020FC6B4D0
:0F0F91000105053B020FE5B40205053B02100404
:100FA000B40305053B021023B40405053B021042BF
:100FB000B40505053B021061B40605053B0210802F
:100FC000753B0002109F74FE7908C293339291D250
:100FD00093D9F7C290D2907908C294A29233D29456
:100FE000D9F7F5692274FD7908C293339291D293AF
:100FF000D9F7C290D2907908C294A29233D294D9F0
:10100000F7F56A2274FB7908C293339291D293D98F
:10101000F7C290D2907908C294A29233D294D9F7B1
:10102000F56B2274F77908C293339291D293D9F772
:10103000C290D2907908C294A29233D294D9F7F593
:101040006C2274EF7908C293339291D293D9F7C28C
:1010500090D2907908C294A29233D294D9F7F56DC8
:101060002274DF7908C293339291D293D9F7C29058
:10107000D2907908C294A29233D294D9F7F56E2215
:1010800074BF7908C293339291D293D9F7C290D2A8
:10109000907908C294A29233D294D9F7F56F227452
:1010A0007F7908C293339291D293D9F7C290D290AC
:1010B0007908C294A29233D294D9F7F57022200E07
:1010C00001229000F2E004126BF7F0C20E22200F12
:1010D00001229000F2E014126BF7F0C20F22200EF2
:1010E00001229000E4123794E004126BABF0C20EC0
:1010F00022200F01229000E4123794E014126BAB0F
:10110000F0C20F22200E01229000E612379BE0046D
:10111000126BBEF0C20E22200F01229000E61237A1
:101120009BE014126BBEF0C20F22200E0122900031
:10113000B2E004126B7FF0122BFAC20E22200F01D4
:10114000229000B2E014126B7FF0122BFAC20F2231
:10115000200E01229000E2E004126B16F0C20E2273
:10116000200F01229000E2E014126B16F0C20F2251
:10117000200E01229000DB123794E004126B6CF019
:10118000C20E22200F01229000DB123794E01412CD
:101190006B6CF0C20F22200E01229000DF123794F8
:1011A000E004126B20F0C20E22200F01229000DF1B
:1011B000123794E014126B20F0C20F22200E01228D
:1011C0009000B6123794E004126B3304126B33F0C4
:1011D000C20E22200F01229000B6123794E01412A2
:1011E0006B3314126B33F0C20F22200E0122E00485
:1011F000126B4604126B46F0C20E22200F0122E051
:1012000014126B4614126B46F0C20F22200E0122FC
:10121000E004126B5904126B59F0C20E22200F0128
:1012200022E014126B5914126B59F0C20F22200ED7
:101230000122E57104126C0AF571C20E22200F0121
:1012400022E57114126C0AF571C20F22200E0122E0
:10125000E004126BD1F0C20E22200F0122E0141222
:101260006BD1F0C20F22200E0122E004126BE4F0D9
:10127000C20E22200F0122E014126BE4F0C20F22F2
:10128000200E0122D210125B95C20E22200F0122E5
:10129000C210125B95C20F22200E0122D216125BE1
:1012A00095C20E22200F0122C216125B95C20F2298
:1012B000E53CB40006053C02132E22B40106053CB1
:1012C00002133822B40206053C02134622B4030678
:1012D000053C02135022B40406053C02135E22B4FE
:1012E0000506053C02136822B40606053C02137687
:1012F00022B40706053C02138022B40806053C020E
:10130000138E22B40906053C02139822B40A06057E
:0E1310003C0213A622B40B06053C0213B022C9
:10131E00B40C06053C0213BE22753C000213C82213
:10132E007A01E55B03FB121440227A01E56203FBAE
:10133E00121440D2B6C2B6227A02E55C03FB121436
:10134E0040227A02E56303FB121440D2B6C2B622E3
:10135E007A03E55D03FB121440227A03E56403FB76
:10136E00121440D2B6C2B6227A04E55E03FB121402
:10137E0040227A04E56503FB121440D2B6C2B622AF
:10138E007A05E55F03FB121440227A05E56603FB3E
:10139E00121440D2B6C2B6227A06E56003FB1214CE
:1013AE0040227A06E56703FB121440D2B6C2B6227B
:1013BE007A07E56103FB121440227A07E56803FB06
:1013CE00121440D2B6C2B622C2B5C2B7C2B67A099C
:1013DE007B007902121440D9FBD2B6C2B67A0A7BD0
:1013EE000F7902121440D9FBD2B6C2B67A0B7B0724
:1013FE007902121440D9FBD2B6C2B67A0F7B0079AD
:10140E0002121440D9FBD2B6C2B67A0C7B01790215
:10141E00121440D9FBD2B6C2B622C2B5C2B7C2B6FA
:10142E007A087B007902121440D9FBD2B6C2B6DA22
:10143E00F122C0E07E028AE07D0820E705C2B502F7
:10144E001452D2B5D2B7C2B723DDEFEBDEEAD0E04D
:10145E00227A0A7B0F1214407A0A7B0F121440D2A2
:10146E00B6C2B62275F00A84AFF0EF2430F02275C2
:10147E00F00A84AFF075F00A84E5F02430F0EF2422
:10148E0030A3F02275F00A84AFF075F00A84243090
:10149E00F0E5F02430A3F0EF2430A3F022126E8F8B
:1014AE001230E81232AB123270200B03123D0620BE
:1014BE00580C12396D1239931239B91239DF1228BC
:1014CE00F112290C123CCF126F8030100612708C64
:1014DE00126FD0126EE7200A03021526C20A3010D0
:1014EE000874FC126C7A0214FF30160574FC126C30
:1014FE007A757E017551001217021217ED12467C95
:10150E001246B71246F2122DFC12478412703F1289
:10151E0070525368E11238BA300C2EC20C301008DB
:10152E0074FA126C7A02153E30160574FA126C7A41
:10153E00755300755200755100D20DC21D757E0196
:10154E0012199712457A123A053007030214AB208E
:10155E000B030215B92008030215B9C20830100892
:10156E0074F8126C7A02157E30160574F8126C7AC5
:10157E00126FFD126FDD126FEE127059127078122B
:10158E003A18200D030215B9301F030215CD127043
:10159E0033127046122340123D06121A49121DFBD9
:1015AE001244421244791244B0C20D301D11121A67
:1015BE0049121DFB1244421244791244B0C21D124C
:1015CE006F1C22F9E573B40117E571B40512E9C277
:1015DE00E7C2E675F00584A8F012160F12163C222B
:1015EE00E922F9E573B40217E571B40612E9C2E710
:1015FE00C2E675F00584A8F012160F12163C22E909
:10160E0022B40003798022B40103794022B402038C
:10161E00792022B40303791022B40403790822B48A
:10162E000503790422B40603790222790122E8B473
:10163E000003896222B40103896322B40203896420
:10164E0022B40303896522896622C21E02165FD266
:10165E001E900088E0C2E7C2E6F57790008AE0703F
:10166E0006122D9302167B122E0602167B90008D0B
:10167E00E0F5782290008AE070201217029000F3B5
:0E168E00E0142490126C7AE577C2E790009881
:10169C00F0126C7AE578126C7AD2652290008FE0A9
:1016AC00F9900090E0FA1217029000F3E0142490E5
:1016BC00126C7AE577900098D2E7F0C2E7126C7A58
:1016CC00E578126C7A9000F3E0142490126C7AE9AD
:1016DC00900099F0126C7AE578126C7A9000F3E035
:1016EC00142490126C7AEA90009AF0126C7AE578D5
:1016FC00126C7AD2652220650122C265900098E0B6
:10170C0020E7199000F3E0142490126C7A90009862
:10171C00E0C2E7126C7A7400126C7A229000F3E04B
:10172C00142490126C7A900098E0C2E7126C7A74D0
:10173C0000126C7A9000F3E0142490126C7A9000F2
:10174C0099E0126C7A7400126C7A9000F3E0142415
:10175C0090126C7A90009AE0126C7A7400126C7A87
:10176C002290008AE070201217ED9000F4E014240F
:10177C0090126C7AE577C2E790009BF0126C7AE5D8
:10178C0078126C7AD2662290008FE0F990008FE08C
:10179C00FA1217ED9000F4E0142490126C7AE577AD
:1017AC0090009BD2E7F0C2E7126C7AE578126C7A63
:1017BC009000F4E0142490126C7AE990009CF012E2
:1017CC006C7AE578126C7A9000F4E0142490126C28
:1017DC007AEA90009DF0126C7AE578126C7AD266F7
:1017EC002220660122C26690009BE020E71990003F
:1017FC00F4E0142490126C7A90009BE0C2E7126C17
:10180C007A7400126C7A229000F4E0142490126C1A
:10181C007A90009BE0C2E7126C7A7400126C7A909A
:10182C0000F4E0142490126C7A90009CE0126C7A14
:10183C007400126C7A9000F4E0142490126C7A907C
:10184C00009DE0126C7A7400126C7A221237AC058F
:10185C00A29000B2E0F99000BD123794E0600A90BB
:10186C0000DB123794E00303034905A2F022123780
:10187C00ACE0F9541F900089F0E954E02323239045
:10188C00008AF0221237AC05A29000DD123794E0EA
:10189C00600A9000DF123794E0540FC4F99000E214
:1018AC00E0540F4905A2F0221237ACE0F9540F9026
:1018BC00008BF0E954F0C490008CF0221237AC0588
:1018CC00A29000A6E00303FA9000E4123794E01211
:1018DC002BAD4A05A2F0221237ACE0FA543F75F05A
:1018EC0003A4240190008DF0EA54C0232390008EB1
:1018FC00F022E573B4010412192822B40203121960
:10190C00EE2212219D9000AFF09000B11218589069
:10191C0000AE1218909000B01218C8229000EBE0A4
:10192C00702F9000E9E0702912219D90014412382B
:10193C001D1237ACF09001C412381D1218589001CA
:10194C000412381D12189090018412381D1218C8F8
:10195C002212219D9000AFF09000B112185B900004
:10196C00AE1218939000B01218CB22E571B4050496
:10197C001219C122121A3622E571B405071219B2D6
:10198C0012170222121A271217ED22E573B4010363
:10199C000219A2B4020F75620075630075640075BC
:1019AC006500756600227940900144E0C2E7C2E60A
:1019BC00F0A3D9F72212170290014412381D1237E6
:1019CC00ACE0C2E7C2E6F02212219D9000ABF09091
:1019DC0000AD12185B9000AA1218939000AC12186C
:1019EC00CB229000ECE0702F9000EAE070291221DD
:1019FC009D90024412381D1237ACF09002C412387C
:0E1A0C001D12185890020412381D12189090E6
:101A1A00028412381D1218C8221219D42279409051
:101A2A000244E0C2E7C2E6F0A3D9F7221217ED900A
:101A3A00024412381D1237ACE0C2E7C2E6F0229027
:101A4A0000EBE0700C9000E9E06003205D03021AED
:101A5A008C9000AFE0201D0630E726021A6B30E6B4
:101A6A0020900088F01215D19000B112187D9000D4
:101A7A00B01218E69000AE1218B712165812168253
:101A8A002222E57EB401349001441237ACE0201DD5
:101A9A000630E726021AA430E620900088F01215D4
:101AAA00D19001C412187A9001841218E3900104AB
:101ABA001218B41216581216822222B40234900155
:101ACA00451237ACE0201D0630E726021ADB30E665
:101ADA0020900088F01215D19001C512187A900151
:101AEA00851218E39001051218B4121658121682BC
:101AFA002222B403349001461237ACE0201D06308E
:101B0A00E726021B1230E620900088F01215D190C9
:101B1A0001C612187A9001861218E390010612186B
:101B2A00B41216581216822222B4043490014712B3
:101B3A0037ACE0201D0630E726021B4930E620902C
:101B4A000088F01215D19001C712187A90018712F5
:101B5A0018E39001071218B412165812168222229C
:101B6A00B405349001481237ACE0201D0630E72650
:101B7A00021B8030E620900088F01215D19001C82F
:101B8A0012187A9001881218E39001081218B412F8
:101B9A0016581216822222B406349001491237AC22
:101BAA00E0201D0630E726021BB730E620900088A9
:101BBA00F01215D19001C912187A9001891218E30E
:101BCA009001091218B41216581216822222B4076A
:101BDA003490014A1237ACE0201D0630E726021B7A
:101BEA00EE30E620900088F01215D19001CA121842
:101BFA007A90018A1218E390010A1218B412165840
:101C0A001216822222B4083490014B1237ACE0201B
:101C1A001D0630E726021C2530E620900088F012C7
:101C2A0015D19001CB12187A90018B1218E390010A
:101C3A000B1218B41216581216822222B4093490C2
:101C4A00014C1237ACE0201D0630E726021C5C303E
:101C5A00E620900088F01215D19001CC12187A90E3
:101C6A00018C1218E390010C1218B41216581216AD
:101C7A00822222B40A3490014D1237ACE0201D06AC
:101C8A0030E726021C9330E620900088F01215D126
:101C9A009001CD12187A90018D1218E390010D125D
:101CAA0018B41216581216822222B40B3490014E1E
:101CBA001237ACE0201D0630E726021CCA30E620A7
:101CCA00900088F01215D19001CE12187A90018EE8
:101CDA001218E390010E1218B41216581216822224
:101CEA0022B40C3490014F1237ACE0201D0630E7C5
:101CFA0026021D0130E620900088F01215D19001CD
:101D0A00CF12187A90018F1218E390010F1218B4AB
:101D1A001216581216822222B40D3490015012372C
:101D2A00ACE0201D0630E726021D3830E620900080
:101D3A0088F01215D19001D012187A9001901218D9
:101D4A00E39001101218B41216581216822222B405
:101D5A000E349001511237ACE0201D0630E72602FE
:101D6A001D6F30E620900088F01215D19001D11233
:101D7A00187A9001911218E39001111218B41216F0
:0F1D8A00581216822222B40F349001521237AC35
:101D9900E0201D0630E726021DA630E620900088C7
:101DA900F01215D19001D212187A9001921218E30B
:101DB9009001121218B4121658121682222290019A
:101DC900531237ACE0201D0630E726021DDA30E653
:101DD90020900088F01215D19001D312187A900141
:101DE900931218E39001131218B41216581216829E
:101DF90022229000ECE0700C9000EAE06003205E83
:101E090003021E3E9000ABE0201D0630E726021EAD
:101E19001D30E620900088F01215F09000AD1218E0
:101E29007D9000AC1218E69000AA1218B712165D40
:101E390012176D2222E57EB401339002441237ACA9
:101E4900E0201D0630E725021E5630E61F90008867
:101E5900F01215F09002C412187A9002841218E355
:101E69009002041218B412165D12176D22B40233CF
:101E79009002451237ACE0201D0630E725021E8C82
:101E890030E61F900088F01215F09002C512187AFA
:101E99009002851218E39002051218B412165D1209
:101EA900176D22B403339002461237ACE0201D06A9
:101EB90030E725021EC230E61F900088F01215F0A7
:101EC9009002C612187A9002861218E3900206123E
:101ED90018B412165D12176D22B40433900247121A
:101EE90037ACE0201D0630E725021EF830E61F90CA
:101EF9000088F01215F09002C712187A9002871222
:101F090018E39002071218B412165D12176D22B465
:101F190005339002481237ACE0201D0630E7250250
:101F29001F2E30E61F900088F01215F09002C8129B
:101F3900187A9002881218E39002081218B412163F
:101F49005D12176D22B406339002491237ACE020B6
:101F59001D0630E725021F6430E61F900088F01245
:101F690015F09002C912187A9002891218E39002AA
:101F7900091218B412165D12176D22B407339002B4
:101F89004A1237ACE0201D0630E725021F9A30E6D9
:101F99001F900088F01215F09002CA12187A900268
:101FA9008A1218E390020A1218B412165D12176DFC
:101FB90022B4083390024B1237ACE0201D0630E7FB
:101FC90025021FD030E61F900088F01215F090020C
:101FD900CB12187A90028B1218E390020B1218B4E4
:101FE90012165D12176D22B4093390024C1237ACE8
:101FF900E0201D0630E72502200630E61F90008804
:10200900F01215F09002CC12187A90028C1218E393
:1020190090020C1218B412165D12176D22B40A330D
:1020290090024D1237ACE0201D0630E72502203C16
:1020390030E61F900088F01215F09002CD12187A40
:1020490090028D1218E390020D1218B412165D1247
:10205900176D22B40B3390024E1237ACE0201D06E7
:1020690030E72502207230E61F900088F01215F043
:102079009002CE12187A90028E1218E390020E1274
:1020890018B412165D12176D22B40C3390024F1258
:1020990037ACE0201D0630E7250220A830E61F9066
:1020A9000088F01215F09002CF12187A90028F1260
:1020B90018E390020F1218B412165D12176D22B4AC
:1020C9000D339002501237ACE0201D0630E725028F
:1020D90020DE30E61F900088F01215F09002D01231
:1020E900187A9002901218E39002101218B412167E
:1020F9005D12176D22B40E339002511237ACE020F5
:0E2109001D0630E72502211430E61F900088E5
:10211700F01215F09002D112187A9002911218E37A
:102127009002111218B412165D12176D22B40F33F4
:102137009002521237ACE0201D0630E72502214AF3
:1021470030E61F900088F01215F09002D212187A2C
:102157009002921218E39002121218B412165D122E
:10216700176D229002531237ACE0201D0630E72589
:1021770002217D30E61F900088F01215F09002D3FF
:1021870012187A9002931218E39002131218B412DD
:10219700165D12176D229000B8E0700E9000BFE038
:1021A70070041221FC221221B52212224322900030
:1021B700A1E0B403030221D64015C39404F90990A2
:1021C70000C1123794E01414900BF4930221E5F93F
:1021D700099000C1123794E01414900BF393232352
:1021E700D9FCF9A2E1E57792E7F577E9A2E0E5778F
:1021F70092E6F57722900097E0B4030302221D4090
:1022070015C39404F9099000B6123794E01414909A
:102217000BDA9302222CF9099000B6123794E014D6
:1022270014900BD9932323D9FCF9A2E1E57792E720
:10223700F577E9A2E0E57792E6F57722E577D2E749
:10224700C2E6F577229000A1E0B4030302226A40B8
:1022570012C39404F9099000C3E01414900BDA93A5
:10226700022276F9099000C3E01414900BD9932346
:1022770023D9FCF9A2E1E57792E5F577E9A2E0E554
:102287007792E4229000A1E0B403030222A940124E
:10229700C39404F9099000C4E01414900BDA930274
:1022A70022B5F9099000C4E01414900BD9932323A5
:1022B700D9FCF9A2E1E57792E5F577E9A2E0E577C0
:1022C70092E4229000A1E0B403030222E84012C383
:1022D7009404F9099000C5E01414900BDA930222D4
:1022E700F4F9099000C5E01414900BD9932323D96E
:1022F700FCF9A2E1E57792E5F577E9A2E0E57792C7
:10230700E422E577D2E5C2E422F5779000BAE070DF
:102317000412224C2212230922F5779000BBE070A9
:102327000412228B2212230922F5779000BCE07059
:10233700041222CA2212230922E573B401030223DD
:102347004FB4020302234F22122D4874009000AFAE
:10235700F09000ABF0C25DC25E1223E412241112AA
:1023670024311224511224711224911224B11224FF
:10237700D11224F11225111225311225511225717E
:102387001225911225B11225D11225F1122611120B
:1023970026311226511226711226911226B11226C3
:1023A700D11226F112271112273112275112277144
:1023B7001227911227B11227D11227F112281112D1
:1023C70028311228511228711228911228B1122887
:1023D700D122E571B40603D25E22D25D22E569F40B
:1023E700547F20E51FE569F4547F30E0182063141B
:1023F7001223D99000B8E0600320200875770012F7
:1024070018FED22022C220C26322E56AF4547F302C
:10241700E0151223D99000B8E060032021087577F2
:10242700051218FED22122C22122E56BF4547F3017
:10243700E0151223D99000B8E060032022087577D1
:102447000A1218FED22222C22222E56CF4547F30EF
:10245700E0151223D99000B8E060032023087577B0
:102467000F1218FED22322C22322E56DF4547F30C7
:10247700E0151223D99000B8E0600320240875778F
:0E248700141218FED22422C22422E56EF45450
:102495007F30E0151223D99000B8E06003202508AD
:1024A5007577191218FED22522C22522E56FF4543C
:1024B5007F30E0151223D99000B8E060032026088C
:1024C50075771E1218FED22622C22622E570F45414
:1024D5007F30E0151223D99000B8E060032027086B
:1024E5007577231218FED22722C22722E569F454F4
:1024F5007F30E1151223D99000B8E0600320280849
:102505007577011218FED22822C22822E56AF454F2
:102515007F30E1151223D99000B8E0600320290827
:102525007577061218FED22922C22922E56BF454CA
:102535007F30E1151223D99000B8E06003202A0806
:1025450075770B1218FED22A22C22A22E56CF454A2
:102555007F30E1151223D99000B8E06003202B08E5
:102565007577101218FED22B22C22B22E56DF4547A
:102575007F30E1151223D99000B8E06003202C08C4
:102585007577151218FED22C22C22C22E56EF45452
:102595007F30E1151223D99000B8E06003202D08A3
:1025A50075771A1218FED22D22C22D22E56FF4542A
:1025B5007F30E1151223D99000B8E06003202E0882
:1025C50075771F1218FED22E22C22E22E570F45402
:1025D5007F30E1151223D99000B8E06003202F0861
:1025E5007577241218FED22F22C22F22E569F454E2
:1025F5007F30E2151223D99000B8E060032030083F
:102605007577021218FED23022C23022E56AF454E0
:102615007F30E2151223D99000B8E060032031081D
:102625007577071218FED23122C23122E56BF454B8
:102635007F30E2151223D99000B8E06003203208FC
:1026450075770C1218FED23222C23222E56CF45490
:102655007F30E2151223D99000B8E06003203308DB
:102665007577111218FED23322C23322E56DF45468
:102675007F30E2151223D99000B8E06003203408BA
:102685007577161218FED23422C23422E56EF45440
:102695007F30E2151223D99000B8E0600320350899
:1026A50075771B1218FED23522C23522E56FF45418
:1026B5007F30E2151223D99000B8E0600320360878
:1026C5007577201218FED23622C23622E570F454F0
:1026D5007F30E2151223D99000B8E0600320370857
:1026E5007577251218FED23722C23722E569F454D0
:1026F5007F30E3151223D99000B8E0600320380835
:102705007577031218FED23822C23822E56AF454CE
:102715007F30E3151223D99000B8E0600320390813
:102725007577081218FED23922C23922E56BF454A6
:102735007F30E3151223D99000B8E06003203A08F2
:1027450075770D1218FED23A22C23A22E56CF4547E
:102755007F30E3151223D99000B8E06003203B08D1
:102765007577121218FED23B22C23B22E56DF45456
:102775007F30E3151223D99000B8E06003203C08B0
:102785007577171218FED23C22C23C22E56EF4542E
:102795007F30E3151223D99000B8E06003203D088F
:1027A50075771C1218FED23D22C23D22E56FF45406
:1027B5007F30E3151223D99000B8E06003203E086E
:0B27C5007577211218FED23E22C23EA2
:1027D00022E570F4547F30E3151223D99000B8E05D
:1027E0006003203F087577261218FED23F22C23FB1
:1027F00022E569F4547F30E4151223D99000B8E043
:1028000060032040087577041218FED24022C240AF
:1028100022E56AF4547F30E4151223D99000B8E021
:1028200060032041087577091218FED24122C24187
:1028300022E56BF4547F30E4151223D99000B8E000
:10284000600320420875770E1218FED24222C2425F
:1028500022E56CF4547F30E4151223D99000B8E0DF
:1028600060032043087577131218FED24322C24337
:1028700022E56DF4547F30E4151223D99000B8E0BE
:1028800060032044087577181218FED24422C2440F
:1028900022E56EF4547F30E4151223D99000B8E09D
:1028A000600320450875771D1218FED24522C245E7
:1028B00022E56FF4547F30E4151223D99000B8E07C
:1028C00060032046087577221218FED24622C246BF
:1028D00022E570F4547F30E4151223D99000B8E05B
:1028E00060032047087577271218FED24722C24797
:1028F00022E573B404012220970F20140B9000935B
:10290000E004126C1DF0D21422C21422900093E055
:10291000B401539007D005A29000607B06120EC44C
:102920003010201210BE1210CE9000F2E09000661F
:1029300012149290079005A29000697B07120EC4B2
:1029400002295D90087305A29000667B06120EC4F2
:1029500090079005A290006C7B04120EC4E573B43E
:102960000303124EF622E573B4030412299E22B427
:10297000040412297A221229C622900096E0B4019A
:10298000041256AA22B407041256D622B40804121E
:10299000571F22B4090412578F22125702229000A7
:1029A00094E0B4010A12509D124EF612505222B415
:1029B000020A124F5B124EF6125052221250F912B6
:1029C0004EF6125052229000B5E0B40107122A468A
:1029D000122A1722B40207122A25122A1722B40338
:1029E00007122A90122A1722B40407122AB1122AB7
:1029F0001722B40507122AD91233BD22B4060712D2
:102A00002B1812340022B40707122A79122A17222F
:102A1000122B39122A172290079005A29000707B82
:102A200010120EC4229007DF05A29000607B0612F0
:102A30000EC412112A12113D122CE305A290006659
:102A40007B0A120EC4229007E505A29000607B0865
:102A5000120EC41211501211609000E2E0FA123608
:102A6000D105A29000687B02120EC490079005A2C7
:102A700090006A7B06120EC4229007D605A2900031
:102A8000607B09120EC41210DE1210F1122BC32249
:102A90009007ED05A29000607B06120EC412117023
:102AA000121183122D0805A29000667B0A120EC433
:102AB000229007FA05A29000607B09120EC4121141
:102AC000961211A99000DF123794E0122D2F05A263
:102AD0009000697B07120EC4229007F305A29000B4
:102AE000607B07120EC49000C11237941211EA9055
:102AF00000C11237941211FB9000C1123794E07597
:102B0000F00284124FCD05A29000697B07120EC41B
:102B1000E990006712147D2290080305A2900060DE
:102B20007B05120EC41211BC1211D3122B4705A241
:102B30009000657B0B120EC42290080D05A2900038
:0E2B4000607B10120EC4229000B6123794E093
:102B4E0075F00284B4010490090022B402049009C5
:102B5E000B22B4030490091622B404049009212216
:102B6E00B4050490092C22B4060490093722B40748
:102B7E000490094222B4080490094D22B40904902D
:102B8E00095822B40A0490096322B40B0490096E0A
:102B9E0022B40C0490097922B40D0390098422B456
:102BAE002B08126F3975F0038422500122126F39EF
:102BBE0075F00384229000E4123794E0B42B0302E4
:102BCE002BEC501A75F003A4240190006912149294
:102BDE0090079005A290006C7B04120EC422900701
:102BEE004405A29000697B07120EC4227B00900060
:102BFE00B2123771B40110755BFF755CFF755DFF26
:102C0E00755EFF755FFF22B40210755BAA755C5589
:102C1E00755DAA755E55755FAA22B40310755B9239
:102C2E00755C49755D24755E92755F4922B404101A
:102C3E00755B88755C11755D22755E44755F8822C3
:102C4E00B40510755BFF755C00755D00755E0075F3
:102C5E005F0022B40610755B82755C41755D207550
:102C6E005E10755F0822B40710755B81755C087580
:102C7E005D40755E04755F2022B40810755B80752B
:102C8E005C10755D02755E40755F0822B4091075A3
:102C9E005B80755C01755D04755E10755F4022B4D6
:102CAE000A10755BAA755C00755D00755E00755F38
:102CBE000022B40B10755B80755C20755D08755E27
:102CCE0002755F0022755B80755C01755D20755E17
:102CDE0000755F08229000B2E014F5F0740AA4901B
:102CEE000AD58582408583417840F5447545007943
:102CFE0044126A338682088683229000DB12379450
:102D0E00E0B401049008CE22B402049008D822B494
:102D1E0003049008E222B404049008EC229008F612
:102D2E00229000DF123794E0B401049008B922B467
:102D3E0002049008C0229008C72230580122206356
:102D4E0008E569F4547F30E516E569F4547F30E008
:102D5E000BD263202005121984D220221219772259
:102D6E007B0012376EF5F0E57784ABF00BF975F05A
:102D7E000CA4FF12376EFB90008BE024182F2B1241
:102D8E006B92F5772290008CE07004122D6E22B4B7
:102D9E000113122DE9F87404C398F8AC77EC28F5FA
:102DAE0077122D6E22B4020E122DE9F8AC77EC28B4
:102DBE00F577122D6E22B403D2122D6E122DE91458
:102DCE00B40008E577C3940CF577221475F00CA4C3
:102DDE002577F57722B40402740022201E06900097
:102DEE00A2022DF59000A3E004122DE3F022740050
:102DFE009000A2F0A3F0222290008AE0B401041207
:102E0E002E7122B40204122F2922B40304122FEFC2
:102E1E0022B40419122D93F575240C122E5B90001A
:102E2E008FF0E575C3940C122E66A3F0221230BDFE
:102E3E00F575240C122E5B90008FF01230BDF575D7
:102E4E002418122E5B900090F0122D9322B47F0363
:102E5E00022E654002E57522B40103022E70500267
:102E6E00E5752290008CE07020AC77EC2402F577AB
:102E7E00122D6E90008FF0EC2404F577122D6E90CB
:102E8E000090F08C77122D6E22B4012D122DE9FDDB
:102E9E007404C39DFDAC77EC24022DF577122D6ED4
:102EAE0090008FF0EC24042DF577122D6E9000908B
:0F2EBE00F0EC2DF577122D6E22B40228122DE9BB
:102ECD00FDAC77EC24022DF577122D6E90008FF06E
:102EDD00EC24042DF577122D6E900090F0EC2DF56D
:102EED0077122D6E22122DE975F00CA4FDAC77EC46
:102EFD002402F577122D6E2DC3940C90008FF0ECFB
:102F0D002404F577122D6E2DC3940C900090F0ECE7
:102F1D00F577122D6E2DC3940CF5772290008CE071
:102F2D007024AC77EC2402F577122D6E90008FF0A3
:102F3D00EC2404F577122D6E900090F08C77122D05
:102F4D006E240CF57722B40131122DE9FD7404C302
:102F5D009DFDAC77EC24022DF577122D6E90008F30
:102F6D00F0EC24042DF577122D6E900090F0EC2DE1
:102F7D00F577122D6E240CF57722B4022C122DE963
:102F8D00FDAC77EC24022DF577122D6E90008FF0AD
:102F9D00EC24042DF577122D6E900090F0EC2DF5AC
:102FAD0077122D6E240CF57722122DE975F00CA4F5
:102FBD00FDAC77EC2402F577122D6E2DC3940C9099
:102FCD00008FF0EC2404F577122D6E2DC3940C9028
:102FDD000090F0ECF577122D6E240C2DC3940CF5AA
:102FED00772290008CE07026AC77EC2402F57712F6
:102FFD002D6E240C90008FF0EC2404F577122D6EBD
:10300D00900090F08C77122D6E240CF57722B40180
:10301D0033122DE9FD7404C39DFDAC77EC24022D14
:10302D00F577122D6E240C90008FF0EC24042DF505
:10303D0077122D6E900090F0EC2DF577122D6E24F9
:10304D000CF57722B4022E122DE9FDAC77EC24029B
:10305D002DF577122D6E240C90008FF0EC24042D9D
:10306D00F577122D6E900090F0EC2DF577122D6EF8
:10307D00240CF57722122DE975F00CA4FDAC77EC3C
:10308D002402F577122D6E240C2DC3940C90008F15
:10309D00F0EC2404F577122D6E2DC3940C90009056
:1030AD00F0ECF577122D6E240C2DC3940CF57722D0
:1030BD007B0012376EFEF5F0E57784FA8E75157587
:1030CD00126F6BFB0BEA75F00CA4FF12376EFB90C1
:1030DD00008BE0240C2F2B126B9C22E56BF4547F9C
:1030ED0030E623C256D25820551BD25543683712AD
:1030FD003284E573B4030412505222B40404125402
:10310D0015221235B422C255C258205638D2564314
:10311D0068205368E87561001238BAE573B403048A
:10312D0012505222B4040412541522123386123452
:10313D008D1234F41235391235844360809000912C
:10314D00E012338A2222E570F4547F30E638D264DF
:10315D00205032D2509007A005A29000507B101243
:10316D000EC47401F5737405F57112325D12199761
:10317D00122BFA1234F412338612348D12353912A1
:10318D00358412328422C25022E56FF4547F30E62A
:10319D0036205132D2519007A005A29000507B10DD
:1031AD00120EC47402F5737406F57112325D1219A4
:1031BD0097122BFA1234F412338612348D123539DC
:1031CD0012358412328422C25122E56EF4547F30BE
:1031DD00E64A205246D2529007B005A29000507B8D
:1031ED0005120EC47441900056F07442900059F0CF
:1031FD00744390005CF0742090005EF07420900099
:10320D005FF07403F57312199712440912443412C6
:10321D003284124EF61253A01253C722C25222E527
:10322D006CF4547F30E626205222D25290009374D3
:0F323D0002F09007C005A29000507B10120EC443
:10324C007404F5731253F012541512328422C252C4
:10325C0022E573B401077431900055F0227432905A
:10326C000055F0222058012212315312319612319E
:10327C00D7200B0312322C22E573B401077568F6C4
:10328C0075610122B402077568F575610222B403F9
:10329C00077568F3756104227568E775611022E59E
:1032AC0073B401041232CA22B402041232CA22B418
:1032BC00030412470F22B404041254232222305860
:1032CC000412359B221232E712331E12335212347F
:1032DC00431234AA12351112355022E56AF4547F88
:1032EC0030E52C204928D2499000B57408F09000A4
:1032FC0091F09000B874FFF09000BF7400F0436040
:10330C00405360CF5367BF436730122A172222C243
:10331C004922E56BF4547F30E529204A25D24A90A6
:10332C0000B57406F0900091F04360205360AF53E9
:10333C0067DF4367509000B87400F09000BF7400D2
:10334C00F02222C24A22E56CF4547F30E529204B4E
:10335C0025D24B9000B57405F0900091F0436010AD
:10336C0053609F5367EF4367609000B87400F09010
:10337C0000BF74FFF02222C24B229000B5E0B408CB
:10338C00104360405360CF5367BF436730122A1716
:10339C0022B4060D4360205360AF5367DF43675080
:1033AC0022B4050C43601053609F5367EF43676072
:1033BC00229000C1123794E01414900BF39305A2E1
:1033CC00790890007023FAA2E0125095F0A3EAD984
:1033DC00F49000C1123794E01414900BF49305A2EE
:1033EC00790890007823FAA2E0125095F0A3EAD95C
:1033FC00F405A2229000B6123794E01414900BD965
:10340C009305A2790890007023FAA2E0125095F06F
:10341C00A3EAD9F49000B6123794E01414900BDAA6
:10342C009305A2790890007823FAA2E0125095F047
:10343C00A3EAD9F405A222E56DF4547F30E52320EC
:10344C004C1FD24C9000DD123794E0600A7400F0EF
:10345C005360F712347F2274FFF04360081234710A
:10346C002222C24C2290082705A29000577B0412FE
:10347C000EC42290079005A29000577B04120EC434
:10348C00229000DD123794E0700A5360F75367F70F
:10349C0012347F224360085367F712347122E56EB1
:1034AC00F4547F30E523204D1FD24D9000BD1237D0
:1034BC0094E0600A7400F05360FB1234E62274FF4F
:1034CC00F04360041234D82222C24D2290081D050C
:1034DC00A290005B7B05120EC42290082205A290DC
:1034EC00005B7B05120EC4229000BD123794E07075
:1034FC000A5360FB5367FB1234E6224360045367A4
:10350C00FB1234D822E56FF4547F30E51D204E19A0
:10351C00D24E9000E9123794E060077400F05367C4
:10352C00FD2274FFF04367022222C24E229000E972
:10353C00123794E070075360FD5367FD2243670216
:10354C005360FD22E570F4547F30E529204F25D2DD
:10355C004F9000EB123794E060077400F05367FE55
:10356C002274FFF0436701E571B4050412170222BF
:10357C001217ED2222C24F229000EB123794E0700A
:10358C00075360FE5367FE224367015360FE22120D
:10359C0035FB12361312362B12364312365B1236AB
:1035AC007312368B1235B4229000B5E0B401077556
:0E35BC00677E75600122B4020775677D756039
:1035CA000222B4030775677B75600422B404077589
:1035DA00677775600822B4050775676F75601022F2
:1035EA00B4060775675F7560202275673F7560408E
:1035FA0022E570F4547F30E50D204F09D24F900038
:10360A00B57401F02222C24F22E56FF4547F30E5EF
:10361A000D204E09D24E9000B57402F02222C24EFD
:10362A0022E56EF4547F30E50D204D09D24D90000D
:10363A00B57403F02222C24D22E56DF4547F30E5C1
:10364A000D204C09D24C9000B57404F02222C24CD1
:10365A0022E56CF4547F30E50D204B09D24B9000E3
:10366A00B57405F02222C24B22E56BF4547F30E593
:10367A000D204A09D24A9000B57406F02222C24AA5
:10368A0022E56AF4547F30E50D204909D2499000B9
:10369A00B57407F02222C249221236C41236D10565
:1036AA00A290006C7B02120EC41236C41237230594
:1036BA00A290006E7B02120EC4229000E2E0C37553
:1036CA00F00C84F9AAF022EAB4000490076222B44A
:1036DA00010490076422B4020490076622B403042A
:1036EA0090076822B4040490076A22B4050490077C
:1036FA006C22B4060490076E22B407049007702265
:10370A00B4080490077222B4090490077422B40A18
:10371A00049007762290077822E9B4000490077A89
:10372A0022B4010490077C22B4020490077E22B4DA
:10373A00030490078022B4040490078222B405048B
:10374A0090078422B4060490078622B407049007DF
:10375A008822B4080490078A22B4090490078C22AC
:10376A0090078E22900089E01475F00AA49009CE81
:10377A008582408583417840F54475450079441235
:10378A006A338682088683EB9322E571B40601A325
:10379A0022E572B4010122B40202A322B40302A3F5
:1037AA00A322C0E005A29000EFE0F5F07410A40592
:1037BA00A28582408583417840F544754500794465
:1037CA00126A338682088683D0E02205A29000A579
:1037DA00E01405A28582408583417840F544754509
:1037EA00007944126A33868208868322C0E005A2E1
:1037FA00900096E0C3940205A285824085834178B1
:10380A0040F5447545007944126A338682088683F6
:10381A00D0E022FFE57E148582408583417840F519
:10382A00447545007944126A338682088683EF22FA
:10383A00E572B4010C9000C605A29000D812386651
:10384A0022B4020C9000CC05A29000D9123866224C
:10385A009000D205A29000DA12386622E0F905A299
:10386A00D90122A302386A9000EFE0B4000D1238A1
:10387A00BA5361FD4368025368E322B4010D12385A
:10388A00BA5361FB4368045368E522B4020D123847
:10389A00BA5361F74368085368E9221238BA536188
:1038AA00EF4368105368F122301F045368E1222263
:1038BA009000F0E020E0065361FD0238CA4361023D
:1038CA0020E1065361FB0238D643610420E2065325
:1038DA0061F70238E243610820E3045361EF2243AF
:1038EA006110229000EFE0F81239657902B80012EF
:1038FA009000F0E030E008E89000EFF0C21F2212DA
:10390A003965B801159000F0E030E10BE89000EF5E
:10391A00F0C21F123A2222123965B802159000F03D
:10392A00E030E20BE89000EFF0C21F123A222212B6
:0E393A003965B803179000F0E030E30BE89019
:1039480000EFF0C21F123A2222123965D9A174037E
:103958009000EFF0D21F1217021217ED2208B804D8
:103968000378002222E56FF4547F30E61B205117BC
:10397800D2519000F0E020E007D2E0F0436102224B
:10398800C2E0F05361FD2222C25122E56EF4547F59
:1039980030E61B205217D2529000F0E020E107D207
:1039A800E1F043610422C2E1F05361FB2222C252DA
:1039B80022E56DF4547F30E61B205317D253900054
:1039C800F0E020E207D2E2F043610822C2E2F053BD
:1039D80061F72222C25322E56CF4547F30E61B20A3
:1039E8005417D2549000F0E020E307D2E3F043618B
:1039F8001022C2E3F05361EF2222C25422740390D2
:103A080000EFF01238ED2058061238711238B22241
:103A18002058061238711238B22220590122C25990
:103A2800791090030405A290031405A2E0A305A24F
:103A3800F0A3D9F6791090030405A290032405A2F7
:103A4800E0A305A2F0A3D9F6791090030405A2908B
:103A5800033405A2E0A305A2F0A3D9F679109003D8
:103A68004405A290035405A2E0A305A2F0A3D9F649
:103A7800791090034405A290036405A2E0A305A26F
:103A8800F0A3D9F6791090034405A290037405A217
:103A9800E0A305A2F0A3D9F6791090038405A290BB
:103AA800039405A2E0A305A2F0A3D9F67910900328
:103AB8008405A29003A405A2E0A305A2F0A3D9F669
:103AC800791090038405A29003B405A2E0A305A28F
:103AD800F0A3D9F6791090010405A290011405A26B
:103AE800E0A305A2F0A3D9F6791090010405A290ED
:103AF800012405A2E0A305A2F0A3D9F6791090014C
:103B08000405A290013405A2E0A305A2F0A3D9F60A
:103B1800791090014405A290015405A2E0A305A2E2
:103B2800F0A3D9F6791090014405A290016405A28A
:103B3800E0A305A2F0A3D9F6791090014405A2905C
:103B4800017405A2E0A305A2F0A3D9F679109001AB
:103B58008405A290019405A2E0A305A2F0A3D9F6DA
:103B6800791090018405A29001A405A2E0A305A202
:103B7800F0A3D9F6791090018405A29001B405A2AA
:103B8800E0A305A2F0A3D9F679109001C405A2908C
:103B980001D405A2E0A305A2F0A3D9F679109001FB
:103BA800C405A29001E405A2E0A305A2F0A3D9F6FA
:103BB80079109001C405A29001F405A2E0A305A222
:103BC800F0A3D9F6791090020405A290021405A278
:103BD800E0A305A2F0A3D9F6791090020405A290FB
:103BE800022405A2E0A305A2F0A3D9F67910900259
:103BF8000405A290023405A2E0A305A2F0A3D9F619
:103C0800791090024405A290025405A2E0A305A2EF
:103C1800F0A3D9F6791090024405A290026405A297
:103C2800E0A305A2F0A3D9F6791090024405A2906A
:103C3800027405A2E0A305A2F0A3D9F679109002B8
:103C48008405A290029405A2E0A305A2F0A3D9F6E8
:103C5800791090028405A29002A405A2E0A305A20F
:103C6800F0A3D9F6791090028405A29002B405A2B7
:103C7800E0A305A2F0A3D9F679109002C405A2909A
:103C880002D405A2E0A305A2F0A3D9F67910900208
:103C9800C405A29002E405A2E0A305A2F0A3D9F608
:103CA80079109002C405A29002F405A2E0A305A22F
:0E3CB800F0A3D9F622123F4012412D124327ED
:103CC6001219B2121A27D25922305801222064083A
:103CD600E569F4547F30E525E570F4547F30E61D40
:103CE600D2642050173064151217021217ED1246CF
:103CF6007C1246B71246F2123CBDD25022C2502266
:103D0600E573B40349123F091241031242FDE56B04
:103D1600F4547F20E63874009000A7F09000A8F0D5
:103D26009000A9F0C25AC25BC25C123D55123DC258
:103D3600123E2F123E9C123F4F123FBC12402912D8
:103D460040961241491241B612422312429022E590
:103D56006AF4547F30E057300B297572019000A544
:103D66007401F0D25A9000BAE0600C20213F7577BA
:103D760000124343D221227577001243431243793E
:103D8600D22122202127D22112468275720190006B
:103D9600A57401F074001245BD9000E6E01250B41F
:103DA60075F008A42407F578124661D26B22C22169
:103DB600200BFA306BF7C26B12468222E56BF45485
:103DC6007F30E057300B297572019000A57403F01F
:103DD600D25A9000BAE0600C20223F757702124357
:103DE60043D22222757702124343124379D222220A
:103DF600202227D2221246827572019000A57403F2
:103E0600F074021245BD9000E6E01250B475F00859
:103E1600A42407F578124661D26C22C222200BFA3E
:103E2600306CF7C26C12468222E56AF4547F30E1A8
:103E360057300B297572019000A57402F0D25A9082
:103E460000BAE0600C20293F757701124343D2295E
:103E560022757701124343124379D229222029275A
:103E6600D2291246827572019000A57402F074017F
:103E76001245BD9000E6E01250B475F008A4240780
:103E8600F578124661D26D22C229200BFA306DF701
:103E9600C26D12468222E56BF4547F30E157300B37
:103EA600297572019000A57404F0D25A9000BAE008
:103EB600600C202A3F757703124343D22A22757776
:103EC60003124343124379D22A22202A27D22A12E6
:103ED60046827572019000A57404F074031245BD04
:103EE6009000E6E01250B475F008A42407F57812A5
:103EF6004661D26E22C22A200BFA306EF7C26E12CB
:103F0600468222206008E569F4547F30E11CE569A9
:103F1600F4547F30E00ED26020280812467C123F0F
:103F260040D2282212467C123F33C2282290030434
:103F360012381D1237AC7400F0227940900304E069
:103F4600C2E5C2E4F0A3D9F722E56AF4547F30E271
:103F560057300B297572029000A57405F0D25B905C
:103F660000BBE0600C20313F757700124385D231EB
:103F7600227577001243851243BBD23122203127A6
:103F8600D2311246BD7572029000A57405F0740018
:103F96001245FB9000E7E01250B475F008A4240720
:103FA600F57812469CD26F22C231200BFA306FF799
:103FB600C26F1246BD22E56BF4547F30E257300BD8
:103FC600297572029000A57407F0D25B9000BBE0E1
:103FD600600C20323F757702124385D23222757704
:103FE600021243851243BBD23222203227D232122A
:103FF60046BD7572029000A57407F074021245FB67
:104006009000E7E01250B475F008A42407F5781282
:0C401600469CD27022C232200BFA30709F
:10402200F7C2701246BD22E56AF4547F30E357307E
:104032000B297572029000A57406F0D25B9000BB4A
:10404200E0600C20393F757701124385D239227521
:1040520077011243851243BBD23922203927D23944
:104062001246BD7572029000A57406F074011245E5
:10407200FB9000E7E01250B475F008A42407F5782D
:1040820012469CD27122C239200BFA3071F7C271EA
:104092001246BD22E56BF4547F30E357300B29758D
:1040A20072029000A57408F0D25B9000BBE0600C35
:1040B200203A3F757703124385D23A22757703126D
:1040C20043851243BBD23A22203A27D23A1246BD46
:1040D2007572029000A57408F074031245FB9000FB
:1040E200E7E01250B475F008A42407F57812469C54
:1040F200D27222C23A200BFA3072F7C2721246BD55
:1041020022206108E569F4547F30E31CE569F45428
:104112007F30E20ED2612038081246B712412DD20A
:1041220038221246B712413CC238227940900344E9
:10413200E0C2E5C2E4F0A3D9F72290034412381D8D
:104142001237AC7400F022E56AF4547F30E4573041
:104152000B297572039000A57409F0D25C9000BC23
:10416200E0600C20413F7577001243C7D2412275AF
:1041720077001243C71243FDD24122204127D24188
:104182001246F87572039000A57409F07400124685
:10419200399000E8E01250B475F008A42407F578CD
:1041A2001246D7D27322C241200BFA3073F7C27380
:1041B2001246F822E56BF4547F30E457300B297530
:1041C20072039000A5740BF0D25C9000BCE0600C0E
:1041D20020423F7577021243C7D2422275770212FC
:1041E20043C71243FDD24222204227D2421246F84E
:1041F2007572039000A5740BF07402124639900098
:10420200E8E01250B475F008A42407F5781246D7F6
:10421200D27422C242200BFA3074F7C2741246F8EA
:1042220022E56AF4547F30E557300B29757203900A
:1042320000A5740AF0D25C9000BCE0600C20493FFB
:104242007577011243C7D249227577011243C7120B
:1042520043FDD24922204927D2491246F8757203FA
:104262009000A5740AF074011246399000E8E01239
:1042720050B475F008A42407F5781246D7D27522F7
:10428200C249200BFA3075F7C2751246F822E56B67
:10429200F4547F30E557300B297572039000A574F2
:1042A2000CF0D25C9000BCE0600C204A3F757703B2
:1042B2001243C7D24A227577031243C71243FDD273
:1042C2004A22204A27D24A1246F87572039000A564
:1042D200740CF074031246399000E8E01250B47581
:1042E200F008A42407F5781246D7D27622C24A20D3
:1042F2000BFA3076F7C2761246F822206208E56998
:10430200F4547F30E51CE569F4547F30E40ED26248
:104312002048081246F2124327D248221246F212CD
:104322004336C248227940900384E0C2E5C2E4F0F9
:10433200A3D9F72290038412381D1237AC7400F00F
:10434200229000E6E01250B4D2E5F5789000EEE05B
:1043520020E0199000EDE020E00C90030412381DDB
:104362001237AC0243719000A70243719000A7E597
:104372007703034578F02205A212231005A2F0125A
:10438200478B229000E7E01250B4D2E5F578900016
:0F439200EEE020E1199000EDE020E10C900344F3
:1043A10012381D1237AC0243B39000A80243B390F8
:1043B10000A8E57703034578F02205A21223200522
:1043C100A2F01247CC229000E8E01250B4D2E5F5F9
:1043D100789000EEE020E2199000EDE020E20C90F0
:1043E100038412381D1237AC0243F59000A9024331
:1043F100F59000A9E57703034578F02205A2122381
:104401003005A2F012480D22755BE0755C62755DA6
:1044110080755E02755FE0756062756202756300AA
:104421007564627565607566027567001248F912F8
:1044310049E32290079005A29000707B10120EC4F0
:10444100229000EEE020E0169000EDE030E0032045
:104451005A0C90030412381D1237AC0244629000CA
:10446100A7E01245A4201D0630E50C02447230E499
:10447100061244E712465E229000EEE020E116901B
:1044810000EDE030E103205B0C90034412381D1273
:1044910037AC0244999000A8E01245E2201D063095
:1044A100E50C0244A930E4061245181246992290FF
:1044B10000EEE020E2169000EDE030E203205C0C1B
:1044C10090038412381D1237AC0244D09000A9E049
:1044D100124620201D0630E50C0244E030E40612AD
:1044E10045491246D422E573B4032B900088E0B409
:1044F1000007436240535BBF22B40107436340534B
:104501005CBF22B40207436220535BDF22B403067F
:10451100436320535CDF22E573B4032B900088E0F2
:10452100B40007435D405364BF22B40107435E40BA
:104531005365BF22B40207435D205364DF22B403F5
:1045410006435E205365DF22E573B4032B90008898
:10455100E0B40007436640535FBF22B401074367DD
:10456100405360BF22B40207436620535FDF22B489
:1045710003064367205360DF22E573B403245362CB
:104581009F53639F435B60435C60535D9F535E9F9A
:1045910043646043656053669F53679F435F604315
:1045A100606022F854C02323900088F01245BDE8D2
:1045B100540F75F008A42407F578E822B400079099
:1045C10000F8E0F57722B401079000F9E0F57722D1
:1045D100B402079000FAE0F577229000FBE0F5774E
:1045E10022F854C02323900088F01245FBE8540FB1
:1045F10075F008A42407F578E822B400079000FCC0
:10460100E0F57722B401079000FDE0F57722B402CE
:10461100079000FEE0F577229000FFE0F57722F8A1
:1046210054C02323900088F0124639E8540F75F0E6
:1046310008A42407F578E822B40007900100E0F50A
:104641007722B40107900101E0F57722B4020790C7
:104651000102E0F57722900103E0F5772212467C12
:104661009000F5E0142490126C7AE57790009EF0AA
:10467100126C7AE578126C7AD2672220670122C225
:10468100679000F5E0142490126C7A90009EE0127D
:104691006C7A7400126C7A221246B79000F6E0141C
:1046A1002490126C7AE57790009FF0126C7AE5788D
:1046B100126C7AD2682220680122C2689000F6E06A
:1046C100142490126C7A90009FE0126C7A7400129C
:1046D1006C7A221246F29000F7E0142490126C7A60
:1046E100E5779000A0F0126C7AE578126C7AD269C5
:1046F1002220690122C2699000F7E0142490126C13
:104701007A9000A0E0126C7A7400126C7A2212483E
:0E4711004E1248871248C012493212496D12EA
:10471F0049A8124A36124EA8124EC2124EDC12523D
:10472F00B31252DC12530512532E12535412537AF2
:10473F00E56BF4547F30E62412513312515312516A
:10474F00731251931251B31251D31251F3125213D8
:10475F00125233125253125273125293229000A4D8
:10476F00E0B2E0F0229000A4E0B2E2F0229000A4C8
:10477F00E0B2E4F0229000A47400F022FF05A290B2
:10478F0000E1E05403700305A222EF30E503024776
:10479F00A620E40305A22212476C30E008EF54C0B4
:1047AF0023230247BFEF54C0232304B40402740031
:1047BF00030354C0CF543FCF4F05A2F022FF05A2F1
:1047CF009000E1E0540C700305A222EF30E50302E4
:1047DF0047E720E40305A22212477430E208EF54A2
:1047EF00C02323024800EF54C0232304B4040274EF
:1047FF0000030354C0CF543FCF4F05A2F022FF0553
:10480F00A29000E1E05430700305A222EF30E503DF
:10481F0002482820E40305A22212477C30E408EF67
:10482F0054C02323024841EF54C0232304B404028D
:10483F007400030354C0CF543FCF4F05A2F022E5BD
:10484F0069F4547F20E12BE569F4547F30E0242094
:10485F00602020201DD2209000E1E030E00AC2E06D
:10486F00F0435B8053627F22D2E0F0436280535B60
:10487F007F2222C220C26022E569F4547F20E32BFD
:10488F00E569F4547F30E22420612020301DD230BE
:10489F009000E1E030E20AC2E2F0435D8053647FB2
:1048AF0022D2E2F0436480535D7F2222C230C26184
:1048BF0022E569F4547F20E52BE569F4547F30E459
:1048CF002420622020401DD2409000E1E030E40A15
:1048DF00C2E4F0435F8053667F22D2E4F0436680E8
:1048EF00535F7F2222C240C262229000E1E020E0AB
:1048FF0009435B8053627F02490F436280535B7FA2
:10490F0020E209435D8053647F0249214364805351
:10491F005D7F20E407435F8053667F2243668053A9
:10492F005F7F22E56FF4547F30E130202E2CD22EA2
:10493F009000947402F09000BAE030E010757201AC
:10494F007400F0435C02124DBB1250522274FFF000
:10495F00535CFD535BE3535CE32222C22E22E56FCF
:10496F00F4547F30E330203E2CD23E9000947402FA
:10497F00F09000BBE030E0107572027400F0435EFF
:10498F0002124E0A1250522274FFF0535EFD535D15
:10499F00E3535EE32222C23E22E56FF4547F30E5FB
:1049AF0030204E2CD24E9000947402F09000BCE058
:1049BF0030E0107572037400F0436002124E59120A
:1049CF0050522274FFF05360FD535FE35360E322B4
:1049DF0022C24E229000BAE030E00C535CFD535BD4
:1049EF00E3535CE30249FF435C02124DBB1250528A
:1049FF009000BBE030E00C535EFD535DE3535EE38C
:104A0F00024A1B435E02124E0A1250529000BCE043
:104A1F0030E00A5360FD535FE35360E322436002CB
:104A2F00124E59125052229000BAE07012124A7F61
:104A3F00124AAD124ADB124B09124B37124B6590DB
:104A4F0000BBE07012124B93124BC1124BEF124C82
:104A5F001D124C4B124C799000BCE07012124CA7F7
:104A6F00124CD5124D03124D31124D5F124D8D2246
:104A7F00E56EF4547F30E02320251FD2259000945B
:0E4A8F007402F09000C6E09000C3F09000D8D2
:104A9D007401F0757201124DBB12505222C22522C3
:104AAD00E56EF4547F30E123202D1FD22D9000941C
:104ABD007402F09000C7E09000C3F09000D874022B
:104ACD00F0757201124DBB12505222C22D22E56DAE
:104ADD00F4547F30E02320241FD2249000947402DC
:104AED00F09000C8E09000C3F09000D87403F0750A
:104AFD007201124DBB12505222C22422E56DF454A4
:104B0D007F30E123202C1FD22C9000947402F09062
:104B1D0000C9E09000C3F09000D87404F0757201E4
:104B2D00124DBB12505222C22C22E56CF4547F3030
:104B3D00E02320231FD2239000947402F09000CA2A
:104B4D00E09000C3F09000D87405F0757201124D1D
:104B5D00BB12505222C22322E56CF4547F30E12364
:104B6D00202B1FD22B9000947402F09000CBE0907C
:104B7D0000C3F09000D87406F0757201124DBB128F
:104B8D00505222C22B22E56EF4547F30E2232035A1
:104B9D001FD2359000947402F09000CCE09000C4C8
:104BAD00F09000D97401F0757202124E0A12505233
:104BBD0022C23522E56EF4547F30E323203D1FD20F
:104BCD003D9000947402F09000CDE09000C4F09000
:104BDD0000D97402F0757202124E0A12505222C29E
:104BED003D22E56DF4547F30E22320341FD2349002
:104BFD0000947402F09000CEE09000C4F09000D9C3
:104C0D007403F0757202124E0A12505222C23422EF
:104C1D00E56DF4547F30E323203C1FD23C9000948B
:104C2D007402F09000CFE09000C4F09000D97404AD
:104C3D00F0757202124E0A12505222C23C22E56CDD
:104C4D00F4547F30E22320331FD23390009474024A
:104C5D00F09000D0E09000C4F09000D97405F0758C
:104C6D007202124E0A12505222C23322E56CF454D3
:104C7D007F30E323203B1FD23B9000947402F090D1
:104C8D0000D1E09000C4F09000D97406F075720266
:104C9D00124E0A12505222C23B22E56EF4547F305E
:104CAD00E42320451FD2459000947402F09000D269
:104CBD00E09000C5F09000DA7401F0757203124EA9
:104CCD005912505222C24522E56EF4547F30E5232D
:104CDD00204D1FD24D9000947402F09000D3E090BF
:104CED0000C5F09000DA7402F0757203124E59127D
:104CFD00505222C24D22E56DF4547F30E4232044FE
:104D0D001FD2449000947402F09000D4E09000C53E
:104D1D00F09000DA7403F0757203124E591250526E
:104D2D0022C24422E56DF4547F30E523204C1FD27E
:104D3D004C9000947402F09000D5E09000C5F09076
:104D4D0000DA7404F0757203124E5912505222C2D9
:104D5D004C22E56CF4547F30E42320431FD2439062
:104D6D0000947402F09000D6E09000C5F09000DA47
:104D7D007405F0757203124E5912505222C243221D
:104D8D00E56CF4547F30E523204B1FD24B900094FB
:104D9D007402F09000D7E09000C5F09000DA740630
:104DAD00F0757203124E5912505222C24B229000CE
:104DBD00D8E0B4010A535BE3535CE3435B0422B4D4
:104DCD00020A535BE3535CE3435C0422B4030A53CE
:104DDD005BE3535CE3435B0822B4040A535BE35388
:104DED005CE3435C0822B4050A535BE3535CE34385
:104DFD005B1022535BE3535CE3435C10229000D9BC
:0E4E0D00E0B4010A535DE3535EE3435D04220B
:104E1B00B4020A535DE3535EE3435E0422B4030A18
:104E2B00535DE3535EE3435D0822B4040A535DE331
:104E3B00535EE3435E0822B4050A535DE3535EE31E
:104E4B00435D1022535DE3535EE3435E10229000FB
:104E5B00DAE0B4010A535FE35360E3435F0422B427
:104E6B00020A535FE35360E343600422B4030A5323
:104E7B005FE35360E3435F0822B4040A535FE353D9
:104E8B0060E343600822B4050A535FE35360E343D6
:104E9B005F1022535FE35360E343601022E56FF42E
:104EAB00547F30E00F20260BD226757201900094B0
:104EBB007401F022C22622E56FF4547F30E20F20FA
:104ECB00360BD2367572029000947401F022C23602
:104EDB0022E56FF4547F30E40F20460BD2467572F7
:104EEB00039000947401F022C24622E572B4011FB4
:104EFB00743C900055F0743E900057F07420900075
:104F0B0058F090005AF090005BF090005DF022B4E6
:104F1B00021F743C900058F0743E90005AF07420BD
:104F2B00900055F0900057F090005BF090005DF012
:104F3B0022743C90005BF0743E90005DF074209006
:104F4B000055F0900057F0900058F090005AF02266
:104F5B009000C312379B12120C9000C312379B1296
:104F6B00121D9000C312379BE0F875F00284124FAC
:104F7B008212383AE8F022FFB40D03024FB14026FB
:104F8B009007F305A29000607B07120EC4EFC39449
:104F9B000D124FCD05A29000697B07120EC4E9904C
:104FAB00006712147D2290080305A29000607B0518
:104FBB00120EC4EF122B5205A29000657B0B120E42
:104FCB00C422B40C03024FD5500590098FF922B4BB
:104FDB001803024FE25008900996C3940CF922B4BF
:104FEB002403024FF2500890099DC39418F922B480
:104FFB00300302500250089009A4C39424F922B440
:10500B003C0302501250089009ABC39430F922B400
:10501B00480302502250089009B2C3943CF922B4C1
:10502B00540302503250089009B9C39448F922B482
:10503B00600302504250089009C0C39454F9229067
:10504B0009C7C39460F9229000C312379BE0141474
:10505B00900BD99305A2790890007023FAA2E01265
:10506B005095F0A3EAD9F49000C312379BE01414C7
:10507B00900BDA9305A2790890007823FAA2E0123C
:10508B005095F0A3EAD9F405A222400374A522742B
:10509B0000229007D605A29000607B09120EC41265
:1050AB0011041211171250C222B41004126F5B229A
:1050BB00500122126F5B229000E612379BE0B41076
:1050CB00030250EB501A75F008A4240790006912E4
:1050DB00149290079005A290006C7B04120EC422D0
:1050EB0090074405A29000697B07120EC42290081A
:1050FB000805A29000607B05120EC49000F81237D1
:10510B00D512124C9000F81237D51212599000F8A4
:10511B001237D5E090006512149290079005A2907B
:10512B0000687B09120EC422E56AF4547F30E01547
:10513B00202111D2217572019000A57401F090000D
:10514B00947403F022C22122E56AF4547F30E115F6
:10515B00202911D2297572019000A57402F09000DC
:10516B00947403F022C22922E56BF4547F30E015CE
:10517B00202211D2227572019000A57403F09000C9
:0E518B00947403F022C22222E56BF4547F30AC
:10519900E115202A11D22A7572019000A57404F034
:1051A9009000947403F022C22A22E56AF4547F30F5
:1051B900E215203111D2317572029000A57405F003
:1051C9009000947403F022C23122E56AF4547F30CE
:1051D900E315203911D2397572029000A57406F0D1
:1051E9009000947403F022C23922E56BF4547F30A5
:1051F900E215203211D2327572029000A57407F0BF
:105209009000947403F022C23222E56BF4547F308B
:10521900E315203A11D23A7572029000A57408F08C
:105229009000947403F022C23A22E56AF4547F3064
:10523900E415204111D2417572039000A57409F05B
:105249009000947403F022C24122E56AF4547F303D
:10525900E515204911D2497572039000A5740AF029
:105269009000947403F022C24922E56BF4547F3014
:10527900E415204211D2427572039000A5740BF017
:105289009000947403F022C24222E56BF4547F30FB
:10529900E515204A11D24A7572039000A5740CF0E5
:1052A9009000947403F022C24A22E570F4547F30CE
:1052B900E01E20271AD2279000EEE030E007C2E076
:1052C900F05362FE22D2E0F043620112467C2222B0
:1052D900C22722E570F4547F30E21E20371AD237F4
:1052E9009000EEE030E107C2E1F05364FE22D2E122
:1052F900F04364011246B72222C23722E570F45402
:105309007F30E41E20471AD2479000EEE030E207D2
:10531900C2E2F05366FE22D2E2F04366011246F27F
:105329002222C24722E570F4547F30E11B202F1757
:10533900D22F9000EDE030E007C2E0F0535CFE228E
:10534900D2E0F0435C012222C22F22E570F4547F9F
:1053590030E31B203F17D23F9000EDE030E107C258
:10536900E1F0535EFE22D2E1F0435E012222C23F08
:1053790022E570F4547F30E51B204F17D24F90007F
:10538900EDE030E207C2E2F05360FE22D2E2F043E0
:1053990060012222C24F229000EEE020E006536213
:1053A900FE0253B043620120E1065364FE0253BC7E
:1053B90043640120E2045366FE2243660122900001
:1053C900EDE020E006535CFE0253D7435C0120E187
:1053D90006535EFE0253E3435E0120E2045360FE7E
:1053E90022436001222222755B02755C02755D020F
:1053F900755E02755F0275600075620575630575F6
:105409006400756500756600756700229007900550
:10541900A29000707B10120EC42212543F12547BCA
:105429001254C41255141255641255B4125604126A
:10543900565412567F22E570F4547F30E01320272A
:105449000FD2279000967401F012545D53627F22A7
:1054590022C2272290082B05A29000607B0A120E17
:10546900C41256B790079005A29000707B10120ED7
:10547900C422E570F4547F30E113202F0FD22F900E
:1054890000967407F012549953627F2222C22F2288
:1054990090087905A29000607B0A120EC41256E3A7
:1054A90090079005A290006D7B03120EC49007909F
:1054B90005A29000707B10120EC422E56FF4547F90
:1054C90030E01D202619D2269000967402F012545D
:1054D900EC9000F3E090006D12149253627F222247
:1054E900C2262290083B05A29000607B0D120EC4D3
:1054F90090084B05A29000707B08120EC49007908B
:0E55090005A29000787B08120EC422E56FF414
:10551700547F30E11D202E19D22E9000967403F08F
:1055270012553C9000F4E090006D12149253627F84
:105537002222C22E2290083B05A29000607B0D120A
:105547000EC490085305A29000707B08120EC490F9
:10555700079005A29000787B08120EC422E56FF42D
:10556700547F30E21D203619D2369000967404F02D
:1055770012558C9000F5E090006D12149253627FE3
:105587002222C2362290083B05A29000607B0D12B2
:105597000EC490085B05A29000707B08120EC490A1
:1055A700079005A29000787B08120EC422E56FF4DD
:1055B700547F30E31D203E19D23E9000967405F0CB
:1055C7001255DC9000F6E090006D12149253627F42
:1055D7002222C23E2290083B05A29000607B0D125A
:1055E7000EC490086305A29000707B08120EC49049
:1055F700079005A29000787B08120EC422E56FF48D
:10560700547F30E41D204619D2469000967406F068
:1056170012562C9000F790006DE012149253627F9F
:105627002222C2462290083B05A29000607B0D1201
:105637000EC490086B05A29000707B08120EC490F0
:10564700079005A29000787B08120EC422E56EF43D
:10565700547F30E01220250ED2259000967408F072
:10566700125671C2172222C2252290088905A290DC
:1056770000607B10120EC422E56EF4547F30E112F5
:10568700202D0ED22D9000967409F012569CC21749
:105697002222C22D229008A905A29000607B101239
:1056A7000EC4221257FF12128012128C1256B72202
:1056B70020100E90087305A290006A7B06120EC494
:1056C7002290083505A290006A7B06120EC42212AA
:1056D70057FF1212981212A41256E32220160E90A8
:1056E700088605A290006A7B03120EC422900883E5
:1056F70005A290006A7B03120EC4221257FF900086
:10570700F31237F61212661212739000F31237F67D
:10571700E090006D121492221257FF12575B20047B
:105727001153627F90079005A29000707B10120EB4
:10573700C42220171143628090089905A290007037
:105747007B10120EC42290074B05A29000757B07B1
:10575700120EC422900096E0B40829E569F4547F3C
:1057670030E02220201ED22090075205A290007020
:105777007B10120EC41202AC1202AC1202ACD2178A
:10578700125A4C2222C220221257FF1257CB200452
:105797001153627F90079005A29000707B10120E44
:1057A700C42220171143628090089905A2900070C7
:1057B7007B10120EC42290074B05A29000757B0741
:1057C700120EC422900096E0B40929E569F4547FCB
:1057D70030E02220201ED22090075205A2900070B0
:1057E7007B10120EC41202AC1202AC1202ACD2171A
:1057F700125A6F2222C22022900096E0B4010412AE
:10580700545D22B402041254EC22B4030412553C32
:1058170022B4040412558C22B405041255DC22B4B8
:10582700060412562C22B4070412549922B4080411
:105837001256712212569C227568201202AC12026F
:10584700AC1202AC1202ACE56BF4547F30E647753C
:10585700680A90065005A29000507B30120EC4E5EE
:105867006FF4547F30E62390068005A29000507BAA
:1058770030120EC41202AC1202AC1202AC1258A7BC
:0E58870012049F125A6F75680022E56DF454EA
:105895007F30E6CD75680022125AF9125B7E756875
:1058A5000022740F9000B2F0A3F074039000B4F0DE
:1058B50074069000B5F074089000B6F0A3F074007B
:1058C5009000B8F0A3F074009000BAF0A3F0A3F034
:1058D50074009000BDF0A3F074009000BFF0A3F039
:1058E50074429000C1F0A3F07404A3F0740EA3F009
:1058F5007442A3F0740479069000C6F02402A3D97B
:10590500FA740E79069000CCF02402A3D9FA7442F9
:1059150079069000D2F02402A3D9FA74019000D838
:10592500F0A3F0A3F074019000DBF0A3F0740090F5
:1059350000DDF0A3F074029000DFF0A3F074159081
:1059450000E1F074009000E2F0A3F0742A9000E406
:10595500F0A3F0740F9000E6F0A3F0A3F0740090AC
:1059650000E9F0A3F074009000EBF0A3F074009050
:1059750000EDF09000EEF074009000EFF0740190EF
:1059850000F0F074789000F2F074019000F3F07478
:1059950002A3F0740AA3F0740AA3F0740AA3F090AA
:1059A50000F87423F09000F97425F09000FA74243F
:1059B500F09000FB7426F09000FC742AF09000FD36
:1059C500742EF09000FE742CF09000FF7433F0906C
:1059D5000100743CF0900101743DF0900102743FA8
:1059E500F09001037440F074007940900144F0A3F5
:1059F500D9FC74007940900244F0A3D9FC74007975
:105A050040900304F0A3D9FC74007940900344F05E
:105A1500A3D9FC74007940900384F0A3D9FC22C279
:105A2500AF79019000F105A290000105A2125ADD9F
:105A3500D2AF22C2AF790190000105A29000F10515
:105A4500A2125B67D2AF22C2AF79129000F205A213
:105A550090000205A2125ADD793F9000B205A2908E
:105A650002D405A2125ADDD2AF22C2AF791290003C
:105A7500F205A290000205A2125ADD798090010478
:105A850005A290001405A2125ADD798090018405C3
:105A9500A290009405A2125ADD798090020405A215
:105AA50090011405A2125ADD798090028405A29016
:105AB500019405A2125ADD79C090030405A2900253
:105AC5001405A2125ADD793F9000B205A29002D4C6
:105AD50005A2125ADDD2AF22E0A343D20205A2F0FD
:105AE500A375D25275D2A2E5D220E0FB53D2FD05B3
:105AF500A2D9E522C2AF791290000205A29000F268
:105B050005A2125B67798090001405A29001040537
:105B1500A2125B67798090009405A290018405A28A
:105B2500125B67798090011405A290020405A21208
:105B35005B67798090019405A290028405A2125BAF
:105B45006779C090021405A290030405A2125B6751
:105B5500793F9002D405A29000B205A2125B67D2EC
:105B6500AF2243D202438E20E0A353D2FD538EDFF2
:105B750005A2F0A305A2D9EA229000B4E020E00531
:105B8500C210025B8CD21020E103C21622D216226B
:105B950020100A9000B4E0C2E0F0025BA99000B4C6
:105BA500E0D2E0F02016089000B4E0C2E1F02290C7
:105BB50000B4E0D2E1F022126E8F12631612633642
:105BC5001263561263761263961263B61263D61287
:105BD50063F6126416126436126456126476126401
:105BE500961264B61264D61264F6126516126536FC
:105BF5001265561265761265961265B61265D6124D
:0E5C050065F61266161266361266561266763E
:105C13001266961266B61266D61266F612671612E8
:105C230067361267561267761267961267B612675F
:105C3300D61267F61268161268361268561268761C
:105C43001268961268B61268D61268F612691612AE
:105C530069361269561269761269961269B6126923
:105C6300D6126A091269F1205F012212708C126F39
:105C7300D0200803025C89C2080551126A21E5514C
:105C8300B4060375510022C2AF790190000005A24A
:105C930090000005A2125ADDD2AF22C2AF79019063
:105CA300000005A290000005A2125B67D2AF90002E
:105CB30000E014F5742290000012126690000012A6
:105CC3001273900000E014F5740490006E12147DBA
:105CD30022756780120F3AE569F4547F30E50D753C
:105CE3006700756280120F2D125CFB22E54EB40330
:105CF300E075670075620022E569F4547F30E01DAA
:105D0300756200125C8A120EB890074005A29000DB
:105D1300667B04120EC41202AC1202AC22125CB9EE
:105D2300025CFB125E0B12629C12616C12624512E2
:105D3300626212627B22E557B40004E8525B22B42C
:105D43000104E9425B22B47E04EA526222B47F0377
:105D5300EB426222E557B40004E8525C22B401042A
:105D6300E9425C22B47E04EA526322B47F03EB422D
:105D73006322E557B40004E8525D22B40104E9420A
:105D83005D22B47E04EA526422B47F03EB426422B0
:105D9300E557B40004E8525E22B40104E9425E22EE
:105DA300B47E04EA526522B47F03EB426522E557D1
:105DB300B40004E8525F22B40104E9425F22B47ED6
:105DC30004EA526622B47F03EB426622E557B4002D
:105DD30004E8526022B40104E9426022B47E04EA7A
:105DE300526722B47F03EB426722E557B40004E80D
:105DF300526122B40104E9426122B47E04EA52688A
:105E030022B47F03EB426822E556B4010B78FE7996
:105E1300017AFE7B01125DEDE556B4020B78FD7944
:105E2300027AFD7B02125DEDE556B4030B78FB7934
:105E3300047AFB7B04125DEDE556B4040B78F77925
:105E4300087AF77B08125DEDE556B4050B78EF7918
:105E5300107AEF7B10125DEDE556B4060B78DF790F
:105E6300207ADF7B20125DEDE556B4070B78FE79CF
:105E7300017AFE7B01125D39E556B4080B78FE7991
:105E8300017AFE7B01125D57E556B4090B78FE7962
:105E9300017AFE7B01125D75E556B40A0B78FE7933
:105EA300017AFE7B01125D93E556B40B0B78FE7904
:105EB300017AFE7B01125DB1E556B40C0B78FE79D5
:105EC300017AFE7B01125DCFE556B40D0B78FD79A7
:105ED300027AFD7B02125D39E556B40E0B78FD792B
:105EE300027AFD7B02125D57E556B40F0B78FD79FC
:105EF300027AFD7B02125D75E556B4100B78FD79CD
:105F0300027AFD7B02125D93E556B4110B78FD799D
:105F1300027AFD7B02125DB1E556B4120B78FD796E
:105F2300027AFD7B02125DCFE556B4130B78FB7941
:105F3300047AFB7B04125D39E556B4140B78FB79C4
:105F4300047AFB7B04125D57E556B4150B78FB7995
:105F5300047AFB7B04125D75E556B4160B78FB7966
:105F6300047AFB7B04125D93E556B4170B78FB7937
:105F7300047AFB7B04125DB1E556B4180B78FB7908
:0E5F8300047AFB7B04125DCFE556B4190B784F
:105F9100F779087AF77B08125D39E556B41A0B7860
:105FA100F779087AF77B08125D57E556B41B0B7831
:105FB100F779087AF77B08125D75E556B41C0B7802
:105FC100F779087AF77B08125D93E556B41D0B78D3
:105FD100F779087AF77B08125DB1E556B41E0B78A4
:105FE100F779087AF77B08125DCFE556B41F0B7875
:105FF100EF79107AEF7B10125D39E556B4200B78FA
:10600100EF79107AEF7B10125D57E556B4210B78CA
:10601100EF79107AEF7B10125D75E556B4220B789B
:10602100EF79107AEF7B10125D93E556B4230B786C
:10603100EF79107AEF7B10125DB1E556B4240B783D
:10604100EF79107AEF7B10125DCFE556B4250B780E
:10605100DF79207ADF7B20125D39E556B4260B7893
:10606100DF79207ADF7B20125D57E556B4270B7864
:10607100DF79207ADF7B20125D75E556B4280B7835
:10608100DF79207ADF7B20125D93E556B4290B7806
:10609100DF79207ADF7B20125DB1E556B42A0B78D7
:1060A100DF79207ADF7B20125DCFE556B42B0B78A8
:1060B100BF79407ABF7B40125D39E556B42C0B782D
:1060C100BF79407ABF7B40125D57E556B42D0B78FE
:1060D100BF79407ABF7B40125D75E556B42E0B78CF
:1060E100BF79407ABF7B40125D93E556B42F0B78A0
:1060F100BF79407ABF7B40125DB1E556B4300B7871
:10610100BF79407ABF7B40125DCFE556B4310B7841
:106111007F79807A7F7B80125D39E556B4320B78C6
:106121007F79807A7F7B80125D57E556B4330B7897
:106131007F79807A7F7B80125D75E556B4340B7868
:106141007F79807A7F7B80125D93E556B4350B7839
:106151007F79807A7F7B80125DB1E556B4360B780A
:106161007F79807A7F7B80125DCF22E556B46B0305
:1061710002617522E557B4002B755B00755C0075F3
:106181005D00755E00755F00756000756100756288
:1061910000756300756400756500756600756700BC
:1061A10075680022B40116755B00755C00755D00B1
:1061B100755E00755F0075600075610022B40213A1
:1061C100756200756300756400756500756600751C
:1061D100670022B4030475680022B4040E9007908E
:1061E10005A29000507B10120EC422B4050E900738
:1061F1009005A29000607B10120EC422B4060E908E
:10620100079005A29000707B10120EC422B40728DB
:1062110090079005A29000507B10120EC490079039
:1062210005A29000607B10120EC490079005A29009
:1062310000707B10120EC422B47E03C27722B47F99
:1062410002D27722E556B46C17E557B40003C25F5A
:1062510022B4010475510022D25F24329000F2F081
:1062610022E556B46713E557B42E0885577F22758A
:106271007F2E2250FA85577F2222E556B46E0DE516
:106281007F70012212628EE55712149222AA7F1AA0
:10629100900050EA700122A3DAFD22E556B43601DE
:1062A1002240FDB467012250FDC39437F91262B553
:1062B100E557F022900050858240858341784089DE
:1062C100447545007944126A33868208868322E543
:1062D100742490126C7AE577126C7A747F126C7A5E
:1062E100E57424B0126C7AE577126C7A747F126CC3
:1062F1007A22E5742490126C7AE577126C7A740034
:0F630100126C7AE57424B0126C7AE577126C7A1C
:106310007400126C7A22E569F4547F30E00C20207E
:10632000087577541262D0D2202230200875775435
:106330001262F3C22022E56AF4547F30E00C20217F
:106340000875774E1262D0D2212230210875774E1F
:106350001262F3C22122E56BF4547F30E00C20225C
:10636000087577481262D0D2222230220875774809
:106370001262F3C22222E56CF4547F30E00C202339
:10638000087577421262D0D22322302308757742F3
:106390001262F3C22322E56DF4547F30E00C202416
:1063A0000875773C1262D0D2242230240875773CDD
:1063B0001262F3C22422E56EF4547F30E00C2025F3
:1063C000087577361262D0D22522302508757736C7
:1063D0001262F3C22522E56FF4547F30E00C2026D0
:1063E000087577301262D0D22622302608757730B1
:1063F0001262F3C22622E570F4547F30E00C2027AD
:106400000875772A1262D0D2272230270875772A9A
:106410001262F3C22722E569F4547F30E10C202890
:10642000087577551262D0D2282230280875775522
:106430001262F3C22822E56AF4547F30E10C20296D
:106440000875774F1262D0D2292230290875774F0C
:106450001262F3C22922E56BF4547F30E10C202A4A
:10646000087577491262D0D22A22302A08757749F6
:106470001262F3C22A22E56CF4547F30E10C202B27
:10648000087577431262D0D22B22302B08757743E0
:106490001262F3C22B22E56DF4547F30E10C202C04
:1064A0000875773D1262D0D22C22302C0875773DCA
:1064B0001262F3C22C22E56EF4547F30E10C202DE1
:1064C000087577371262D0D22D22302D08757737B4
:1064D0001262F3C22D22E56FF4547F30E10C202EBE
:1064E000087577311262D0D22E22302E087577319E
:1064F0001262F3C22E22E570F4547F30E10C202F9B
:106500000875772B1262D0D22F22302F0875772B87
:106510001262F3C22F22E569F4547F30E20C20307E
:10652000087577561262D0D230223030087577560F
:106530001262F3C23022E56AF4547F30E20C20315B
:10654000087577501262D0D23122303108757750F9
:106550001262F3C23122E56BF4547F30E20C203238
:0365600008757744
:106563004A1262D0D2322230320875774A1262F36D
:10657300C23222E56CF4547F30E20C203308757785
:10658300441262D0D233223033087577441262F357
:10659300C23322E56DF4547F30E20C203408757762
:1065A3003E1262D0D2342230340875773E1262F341
:1065B300C23422E56EF4547F30E20C20350875773F
:1065C300381262D0D235223035087577381262F32B
:1065D300C23522E56FF4547F30E20C20360875771C
:1065E300321262D0D236223036087577321262F315
:1065F300C23622E570F4547F30E20C2037087577F9
:106603002C1262D0D2372230370875772C1262F3FE
:10661300C23722E569F4547F30E30C2038087577DC
:10662300571262D0D238223038087577571262F386
:10663300C23822E56AF4547F30E30C2039087577B9
:10664300511262D0D239223039087577511262F370
:10665300C23922E56BF4547F30E30C203A08757796
:106663004B1262D0D23A22303A0875774B1262F35A
:10667300C23A22E56CF4547F30E30C203B08757773
:10668300451262D0D23B22303B087577451262F344
:10669300C23B22E56DF4547F30E30C203C08757750
:1066A3003F1262D0D23C22303C0875773F1262F32E
:1066B300C23C22E56EF4547F30E30C203D0875772D
:1066C300391262D0D23D22303D087577391262F318
:1066D300C23D22E56FF4547F30E30C203E0875770A
:1066E300331262D0D23E22303E087577331262F302
:1066F300C23E22E570F4547F30E30C203F087577E7
:106703002D1262D0D23F22303F0875772D1262F3EB
:10671300C23F22E569F4547F30E40C2040087577CA
:10672300581262D0D240223040087577581262F373
:10673300C24022E56AF4547F30E40C2041087577A7
:10674300521262D0D241223041087577521262F35D
:10675300C24122E56BF4547F30E40C204208757784
:106763004C1262D0D2422230420875774C1262F347
:10677300C24222E56CF4547F30E40C204308757761
:10678300461262D0D243223043087577461262F331
:10679300C24322E56DF4547F30E40C20440875773E
:0C67A300401262D0D244223044087577C6
:1067AF00401262F3C24422E56EF4547F30E40C20B1
:1067BF00450875773A1262D0D24522304508757771
:1067CF003A1262F3C24522E56FF4547F30E40C2095
:1067DF0046087577341262D0D24622304608757754
:1067EF00341262F3C24622E570F4547F30E40C2079
:1067FF00470875772E1262D0D24722304708757737
:10680F002E1262F3C24722E569F4547F30E50C2063
:10681F0048087577591262D0D248223048087577E8
:10682F00591262F3C24822E56AF4547F30E50C2016
:10683F0049087577531262D0D249223049087577CB
:10684F00531262F3C24922E56BF4547F30E50C20FA
:10685F004A0875774D1262D0D24A22304A087577AE
:10686F004D1262F3C24A22E56CF4547F30E50C20DE
:10687F004B087577471262D0D24B22304B08757791
:10688F00471262F3C24B22E56DF4547F30E50C20C2
:10689F004C087577411262D0D24C22304C08757774
:1068AF00411262F3C24C22E56EF4547F30E50C20A6
:1068BF004D0875773B1262D0D24D22304D08757757
:1068CF003B1262F3C24D22E56FF4547F30E50C208A
:1068DF004E087577351262D0D24E22304E0875773A
:1068EF00351262F3C24E22E570F4547F30E50C206E
:1068FF004F0875772F1262D0D24F22304F0875771D
:10690F002F1262F3C24F22E56BF4547F30E60C2056
:10691F0052087577291262D0D252223052087577F9
:10692F00291262F3C25222E56CF4547F30E60C2038
:10693F0053087577281262D0D253223053087577D7
:10694F00281262F3C25322E56DF4547F30E60C2017
:10695F0054087577271262D0D254223054087577B5
:10696F00271262F3C25422E56EF4547F30E60C20F6
:10697F0055087577261262D0D25522305508757793
:10698F00261262F3C25522E56FF4547F30E60C20D5
:10699F0056087577251262D0D25622305608757771
:1069AF00251262F3C25622E570F4547F30E60C20B4
:1069BF0057087577241262D0D2572230570875774F
:1069CF00241262F3C2572220970C20140875775AAD
:1069DF001262D0D2142230140875775A1262F3C2A1
:1069EF001422200E0122E57424B0126C7A746812FE
:0969FF006C7A7401126C7AC20E6C
:106A080022200F0122E57424B0126C7A7468126C8B
:106A18007A7441126C7AC20F22E57424B0126C7A2F
:106A2800746A126C7AE551126C7A22E627F52F08FF
:106A380009E637F530782F22C3E697F52F0809E6DF
:106A480097F530782F22862F8731080986308732CC
:106A5800126AD37834228634088635088636088642
:106A6800378731098732126A76782F793622753856
:106A780000753910126AB8126A89126AACD539F4ED
:106A880022C3E5369531E5379532E5389400500153
:106A980022E5369531F536E5379532F537E5389400
:106AA80000F53822B3E52F33F52FE53033F53022E2
:106AB800C3E53433F534E53533F535E53633F536A6
:106AC800E53733F537E53833F53822E52F8531F0EA
:106AD800A4F53485F035E5308532F0A4F53685F037
:106AE80037E5308531F0A42535F535E53635F0F54F
:106AF80036E5373400F537E52F8532F0A42535F52E
:106B080035E53635F0F536E5373400F53722B40B80
:106B18000122500122740022B401012250037401A1
:106B280022B4030122500122740322B4020122502C
:106B380003740222B41A0122500122741A22B402E8
:106B480001225003740222B4D8012250012274D8C1
:106B580022B40201225003740222B4F2012250012D
:106B68002274F222B40101225003740122B40501F7
:106B780022500122740522B401012250037401221B
:106B8800B41A0122500122741A22B47F0122500142
:106B980022747F22B47F0122500122126ED2543F08
:106BA800241F22B40101225003740122B42B0122B4
:106BB800500122742B22B40101225003740122B423
:106BC800100122500122741022B4010122500374D2
:106BD8000122B47F0122500122747F22B4010122D4
:106BE8005003740122B4100122500122741022B4FF
:106BF8000A01225003740A22B4E6012250012274C9
:106C0800E622B40501225003740522B4060122507D
:106C18000122740622B40003740222B40302740130
:106C28002243B71843B812758790758922758DFC71
:106C3800758BFCD28E759850C299C298D2ACC2029C
:106C4800758CB0758AB075470475480575493275F5
:106C58004C02754D0390FC188582CA8583CB8582CA
:106C6800CC8583CDC20643C804D28CD2A9D2ADD27A
:106C7800AF22D202F5992002FD22C0E0C0D0E9C0BF
:106C8800E0E582C0E0E583C0E0309914C202C29911
:106C9800D0E0F583D0E0F582D0E0F9D0D0D0E03272
:106CA800309807C298E599126E67D0E0F583D0E076
:106CB800F582D0E0F9D0D0D0E032B4F8083007023D
:106CC800C207D20822B4FA10E573B4040122D2072D
:106CD800D20BD20C43680122B4FC13D20AC20BC2F5
:106CE800085361FE5368FE12199712457A22B4FBC5
:106CF80009D207D20BD20C4368012220770122B4B3
:106D0800F812E57424B0126C7A7469126C7A740300
:106D1800126C7A22B4FA12E57424B0126C7A74698F
:106D2800126C7A7401126C7A22B4FC12E57424B0E5
:106D3800126C7A7469126C7A7400126C7A22B4FB41
:106D480011E57424B0126C7A7469126C7A740212A8
:106D58006C7A22B4F00775580075590022B4F1070F
:106D680075580075590022B4F20775580075590016
:0F6D780022B4F31D75580075590022F99000F1EF
:106D8700E0B4010930100122E9126CC222E9126D48
:106D9700032250E8F99000F1E0B4010122E57424E0
:106DA70090F57BE9B57B08755801C211C21822E539
:106DB700742480F57BE9B57B08755901D211C21897
:106DC70022E57424B0F57BE9B57B06755801D21826
:106DD7002230E70D75580075590022026E21026EA8
:106DE700382018FA2011F4A958B9000122A958B976
:106DF70001060558C3F55422B9020C0558F555602C
:106E070003D21322D21322B903060558C3F554221D
:106E1700B90406755801026E0422A959B900012266
:106E2700A959B901080559C3F554D2132275590157
:106E370022A958B9000122A958B901050558F556E4
:106E470022B9020A0558F557125D26D21322B90353
:106E5700050558F55622B90406755801026E4D22EC
:106E6700F57C900082E0B4000122900080E0900061
:106E770001F582E57CF0900080E004B43F027400E5
:106E8700F0900082E014F022C2AC900082E0B43EA1
:106E970003D2AC2204F0900081E0900001F582E07B
:106EA700F57D900081E004B43F027400F0D2ACE5B8
:106EB7007D126D5B9000F1E0B40107200803026EBC
:106EC7008F22026E8F3013C0C21322900083E0041A
:106ED700B410027400F0900040A98229F582E022E4
:106EE700900087E0FA900084E004B40F0274FFF08A
:106EF700900540932A900087F0900086E004B41034
:106F0700027400F0F9900087E0FA900040E58229CA
:106F1700F582EAF022900087E0FA900085E004B459
:106F2700110274FFF090054F932A900087F0126FBB
:106F37000022126ED254016008126ED2541F2460D0
:106F470022747F22126ED2541F242822126ED2542A
:106F57003F241422126ED254016006126ED2540FCF
:106F670022740C227C04DC0122126ED2540FB575F8
:106F77000122500122026F6D22E573B40401223011
:106F8700580122E569F4547F20E518E570F4547F31
:106F970030E61120640D30100A200907B20B126F7A
:106FA700B0D20922C209C26422300B0AD207D20B1F
:106FB700436801D20C22D20AC20BC2085361FE53A6
:106FC70068FE12199712457A22300609C206300761
:106FD70002C207D208220553E553B460097553006E
:106FE7001238ED123A18220552E552B40C0122B4B8
:106FF7001803755200220551E551B40612C21DE56A
:107007007E04B411027401F57E755100D20D22B4CD
:10701700020712199712457A22B4030612457AD24B
:107027001D22B4050612199712457A229000A1E095
:1070370004B408027400F02274079000A1F02290B3
:107047000097E004B408027400F0227407900097D8
:10705700F02230580122E553B4000122E552B40072
:107067000443610122B406045361FE22B4030122E2
:107077002230580122E553B4000443680122B406C4
:10708700035368FE229000F2E0F5757540197541CB
:10709700F57542007543007840857544754500795C
:0C70A70044126A5E864F08E604F5502291
:00000001FF
